:040000006F30B0604D
:100004000000000000000000243B0000443B00000E
:1000140000000000083E0000000000000000000096
:10002400083E0000083E0000000000000000000040
:100034008832000000000000900200000000000070
:10004400083E0000083E0000083E0000083E000094
:10005400083E0000083E0000F0360000183700009B
:10006400403700006837000090370000083E000069
:10007400083E0000083E0000083E0000083E000064
:10008400083E0000083E0000083E0000083E000054
:10009400083E0000083E0000083E0000B83700009B
:1000A400083E0000083E0000083E0000083E000034
:1000B400083E0000083E0000083E0000083E000024
:1000C400083E0000083E0000083E0000083E000014
:1000D400083E0000DE3A00007E5B0000C65B0000C4
:1000E40030380000083E0000083E0000083E0000D2
:1000F400083E0000083E0000083E0000083E0000E4
:1001040000000000083E0000083E0000083E000019
:100114000E5C0000565C0000083E0000083E000033
:10012400083E0000083E0000083E0000083E0000B3
:10013400083E0000083E0000083E0000083E0000A3
:10014400083E0000083E0000083E0000083E000093
:10015400083E0000083E0000083E0000925C0000DB
:10016400DA5C0000225D0000083E0000083E00004A
:10017400083E0000083E0000083E0000083E000063
:10018400083E0000083E0000083E0000083E000053
:10019400083E0000083E0000083E0000083E000043
:1001A400000000000000000000000000000000004B
:0C01B4000000000000000000000000003F
:1001C00097020120938202E4938202E0739002344A
:1001D00003210500224573100530B1A819712320B1
:1001E000250006C006C216CAF322003093F2820030
:1001F000638402009302000816C412C81ACC1ECEF3
:1002000022D026D22AD42ED632D836DA3ADC3EDEB6
:10021000C2C0C6C2CAC4CEC6D2C8D6CADACCDECE26
:10022000E2D0E6D2EAD4EED6F2D8F6DAFADCFEDE96
:1002300003A1050009A002457310153492403785CB
:10024000000013050580732005302245732005301A
:100250004242D2426243F243025492542255B25572
:100260004256D2566257F257064896482649B64932
:10027000464AD64A664BF64B065C965C265DB65DF2
:10028000465ED65E665FF65F09617300203000004F
:10029000197116CA9302000816C49302000273A0D3
:1002A000428006C212C81ACC1ECE22D026D22AD430
:1002B0002ED632D836DA3ADC3EDEC2C0C6C2CAC456
:1002C000CEC6D2C8D6CADACCDECEE2D0E6D2EAD4E6
:1002D000EED6F2D8F6DAFADCFEDE73110134EF0066
:1002E000F006EF10703AEF005009731101341384D7
:1002F0008189032904006304090223200400732573
:1003000010342AC013840189044023A024001384DC
:100310004189044003A10400024573101534924042
:10032000B78200009382028073A00230A24273A0C1
:1003300002304242D2426243F24302549254225566
:10034000B2554256D2566257F25706489648264949
:10035000B649464AD64A664BF64B065C965C265D25
:10036000B65D465ED65E665FF65F0961730020305B
:100370000000397101436EC619A0397141536AC832
:1003800066CA62CC5ECE19A0397101535AD056D2DA
:1003900052D44ED64AD826DA22DC06DE330161403A
:1003A000828241114AC026C222C406C68282B24D50
:1003B0004101024D924C224CB24B4101024B924AF8
:1003C000224AB2494101024992442244B2404101C9
:1003D00082803D432A876373C3029377F700BDEFA2
:1003E000ADE5937606FF3D8ABA960CC34CC30CC7A5
:1003F0004CC74107E36BD7FE11E28280B306C340CE
:100400008A069702000096966780A6002307B70029
:10041000A306B7002306B700A305B7002305B7005E
:10042000A304B7002304B700A303B7002303B70056
:10043000A302B7002302B700A301B7002301B7004E
:10044000A300B7002300B700828093F5F50F9396C1
:100450008500D58D93960501D58D61B793962700BC
:100460009702000096968682E78086FA9680C117EA
:100470001D8F3E96E374C3F8A5B703A581808280E3
:10048000EFF23FF2938781809843050798C3EF10FE
:10049000E0623C45FD173CC589E77C413CC5EF1057
:1004A000A066EF10D01105B7634205029307803EA6
:1004B0003347F5023365F5023305F5021305753E42
:1004C0003345F5023307F7023A9582807D558280E5
:1004D00001458280014582800145828001458280FC
:1004E000EFF23FEC1D649D641304846D9384446EAD
:1004F00063639400C9BD1C4011048297D5BFEFF21D
:100500005FEA1D649D641304446E9384C46E636348
:10051000940055BD1C4011048297D5BFEFF27FE8CF
:10052000F93FEF30206445B5EFF2BFE7B7050000B3
:1005300037650000D1471547930600200146938593
:10054000C5511305C5EEEF10C057EF10406FA5BDA4
:10055000EFF23FE5EF103014EF20104CEF00905C0D
:10056000EF10700DEF102029C137EF10700D192C0E
:10057000EF10402B014581BDEFF2BFE2D13F0145B5
:1005800099B5EFF27FE0AA89EF10405319C1EF103F
:10059000603B2545EF10C0114441130445006396AC
:1005A0008400EF10A051014919A8138944FF214686
:1005B000CE854A85EF00301401E9EF10205019C1B3
:1005C000EF10A0394A85DDBB8440D1BF09E57D55D8
:1005D00082807D55CDBBEFF2DFDC2A842E85328907
:1005E000AE8445377DF522852686A545EF10E00EC1
:1005F0000145231C2401230E0400231D0400D9BF40
:10060000EFF23FDA1E2D41112A84C18B9DE71C5564
:100610008DC32EC68297AA84B24501CD2A8637653E
:100620000000A285130545EFEF00504926854101E2
:1006300059BB1E2C93E707011EAC1E2CA18B89C74A
:100640003E2CE554A18BFDF35C5489CF2285829723
:10065000AA8405E13E2C93E787003EAC5C2C85071D
:100660005CACE9B785679387F7F0FD8D2EAC8144CC
:10067000D5B7E957E31CF5FAF1BF5C2D85CBEFF256
:100680005FD2FD1793F7F70F5CAD2A84014789EF1E
:100690001C5989E70147231D040039A082972A8746
:1006A00075D9E957E309F5FE3A8531BB7D573A859F
:1006B0008280EFF21FCF582D11E77D55EF000067C4
:1006C000014521A05C5999C38297F5B96955FDB7D9
:1006D000EFF23FCD582D11E77D55EF002065014524
:1006E00021A01C5D99C38297F9B96955FDB70CD15A
:1006F00001458280EFF25FC993894186854A83A7CD
:10070000418663863705EF10007983A741862A8AE0
:10071000638D370303A441865C4018401309C4FE6F
:100720005CC398C340C000C0EF10C0217C5099C387
:100730004A8582974A85EF10800B631B55014A85D5
:10074000EF00907FEF1060215285EF108075BDB1F2
:10075000EF10A0205285EF10C0744848EF00B06A37
:100760004A85EF10A00561BFEFF2BFC31384019764
:10077000130904011C4091C382971104E31C24FF58
:10078000953FEDB7EFF2FFC137060000B7650000F7
:10079000930800023D489307002013870198814683
:1007A000130686769385C5F21385018FEF10E02D31
:1007B0001385018FEF10A04839B1EFF29FBE2A8454
:1007C000FD541C406314F4000145F5BEEF10A06C0D
:1007D0002A89084044CD3115EF10A0414A85EF1019
:1007E000406CC5B7EFF2FFBB41112A842E8532C69B
:1007F0002EC4EF1080363246A24519C68547630DD8
:10080000F60001454101C1B65840938745011CC31C
:1008100098CD5CC0C0C9F5B71C406388870083C60B
:10082000550303C7170263FAE600D4431387450153
:1008300098C294CDD8C3DCC9E9B79C43F9BFEFF2A5
:100840005FB64111B2842E8689452A8436C6EF00F0
:10085000D068B246930744011CCC5CC846AC14B4C3
:10086000014541018DB6EFF23FB283A701854111E9
:100870002EC62A8491C38297EF10E0615E2CAA896C
:1008800089CFFD175EACEF10C06183A7C18401451D
:1008900091CB22858297014531A0B24791E7EF10B5
:1008A00040607955410119BEEF104021232805020F
:1008B0001034AA85AA84130544012D37B247635C1E
:1008C000F0001389C404700081454A85EF10A04BE5
:1008D0004A85EF1020404E85EF10A05CEF00507766
:1008E000885845D5C1B7EFF2DFAB83A781842A844E
:1008F00091C38297EF10205AAA8448489307440175
:10090000630EF5003115EF10C02E05442685EF105B
:10091000405919C0EF00D073014575B45E2C8507AE
:100920005EAC0144E5B7EFF2DFA72A8451057135CB
:10093000484CEF00504D2285EF005068014561B4EE
:10094000EFF23FA64111AE84AA85194532C636C4DE
:10095000EF0070612A841DC9A246930745011CCD92
:1009600014B55CC932461385340071994205418142
:1009700032B042060AB0418211053305C502EF00CC
:10098000903348CC19E52285793F01442285410105
:100990001DBC36302324040223260402232804022B
:1009A00001476345D70023120402CDB71E3010580B
:1009B0009107B387E7020507AA9790C31CD8D5B75C
:1009C0001E3163EEC706EFF23F9C83A781842A8421
:1009D0003289AE8991C38297EF10E04B045891E4BD
:1009E000EF10204C75556FF07F9D9C401CD8EF1088
:1009F000404B4A86CE8523A0040013854400C92EAF
:100A0000EF1060495C542A8991C384C31C5444D4B8
:100A100091E304D45E304848510485071EA8630C56
:100A200085003115EF10E01C4A85EF108047EF007C
:100A3000306201454DBF4A85EF10A046DDBF7D55B0
:100A40008280EFF29F9341112A842E8B328A36C620
:100A5000EF10C00683A701852A8999C32285829752
:100A6000EF1060435E30AA89639C070CB247814453
:100A70006399070CEF10E042795541016FF07F93C5
:100A8000B2472328090281EB4E85EF108041F957C8
:100A90002328F902D5B71034CA855E85A133B24741
:100AA000635DF000EFF07F9DAA847000814556855C
:100AB000EF10602D5685EF10E0214E85EF10603E5F
:100AC000EF001059032509034DF9EF10C03CB24760
:100AD000AA89268C635DF000EFF03F9AB247330C91
:100AE0009540A6973385A740634A05042AC6E28449
:100AF0005E30D9D70454984018D4585463149700E2
:100B000023260402FD175EB04E85EF1080391230A7
:100B10006373CA005286938544005A85552CEF10A2
:100B200080371C589CC004D8EF10A03783A7C1841D
:100B30000145A1D722858297014581B702C645BFED
:100B40008144930B4401930AC9045DB7EFF27F859A
:100B50004111EF104034138741811C23850793F71F
:100B6000F70F1CA383A7C18081C72AC6829732458D
:100B7000EF10203341016FF01F85EFF29F8241118A
:100B8000EF106031138741811C23FD1793F7F70F96
:100B90001CA383A7018181C72AC682973245EF1023
:100BA000403041016FF03F8203C5418182809378DC
:100BB00008044111639E080099689388880D937317
:100BC0000801638B03001378E8FF930E000219A855
:100BD000996893884803E5B713731800930E0003D0
:100BE000E30503FE13732800630E03066358060231
:100BF0003306C0409302D0020A8E814F294F63957D
:100C0000E6073373D6023356D602469303430300F6
:100C1000850F050EA30F6EFE7DF20DA01373480025
:100C20009302B0026317030093728800B33250003E
:100C3000960279F2930600035480854FFE8663D3B3
:100C4000FF00BE8613781801158F631308046385AF
:100C500002006353E0007D172A86B308E500130302
:100C6000000221A88142F1B71373F600118271BF0F
:100C70006374B6002300660005063388C840E34964
:100C800000FF3A866353070001467D173295118FA6
:100C9000638802006374B500230055007D170505C5
:100CA00063870302AA96130800031DA86374B600A5
:100CB0002300D60105063388C840E34900FF3A8681
:100CC0006353070001467D173295118FE1BF2A86D5
:100CD000B308E500CDB76374B50023000501050531
:100CE0003386A640E3C9CFFEFD56FD1F6383DF00B8
:100CF00099E7AA873306E5001308000231A8637656
:100D0000B5003306F101102210A10505F9BF63F407
:100D1000B700238007018507B306F640E349D0FEFC
:100D20006353070001473A9541018280EFF26FE774
:100D30002A849D3D09C523AC81806FF0CFE8EF0088
:100D4000F05775D900D9D5BF0D47AA876376C7007C
:100D50009377350091C7AA873E966397C70682802E
:100D600093F7F50F13978700D98F139707015D8FBE
:100D7000B308C500AA87BD463388F84063EB060375
:100D800093574600C156B386D7029207AA970D48DB
:100D900036963383C700BE86B308D3406362180318
:100DA00013572600F156B306D7020A07BA973696AC
:100DB00065B798C3D8C398C7C10723AEE7FE6DBF18
:100DC000910623AEE6FEC9BF8507A38FB7FE71B7B4
:100DD0003D47AA876377C700B367B5008D8BA5CB66
:100DE000AA8701476315C708828003A80700C107C7
:100DF0004107232807FF03A847FF232A07FF03A86B
:100E000087FF232C07FF03A8C7FF232E07FF338884
:100E1000F840E3EC06FD9356460013974600B307EF
:100E2000E500BA954157B386E602014736968D46EE
:100E30003308E64063C306031357260093162700C2
:100E4000B697B695F1563307D7023A9659BFAE8793
:100E50002A87B388C500BD465DBF3388E500832877
:100E600008003388E700110723201801D1B7B386A3
:100E7000E50003880600B386E70005072380060126
:100E800095B763F2A504B386C500637ED50293458A
:100E9000F6FF8147FD176393F50082803387F600E4
:100EA000030807003387C7002A9723000701DDB72F
:100EB0003387F500830607003307F500850714A381
:100EC000E318F6FE82808147E5BF0DC6AA87850537
:100ED0000387F5FF85079306F6FFA38FE7FE09EB6F
:100EE0003E9685076393C7008280A38F07FED5BF18
:100EF0003686F1FE828001476314E600814739A8F7
:100F0000B307E50083860700B387E5009C23B3871A
:100F1000F640E207E18799E30507F9FE3E85828006
:100F2000AA870387070001E73385A74082808507EA
:100F3000CDBFEFF28FC42E89B30B250141112A8C4E
:100F4000B68563F5AB001349F5FFFD5BC169376AF0
:100F500000006284930AB002130B0002FD19130A09
:100F60000A0D31A8130750026389E7026373740105
:100F70001CA013051400B284138614002A8483076E
:100F80000600EDF363060900637C742F2300040060
:100F90003305844141016FF0CFC101481307D002EE
:100FA000930630021305000331A0639E57011368B6
:100FB000480026868307160093041600E397E7FE91
:100FC00013680801FDB76395670113688800D5B7FA
:100FD0006395D70013680802E9BF6395A7001368FB
:100FE0001800C1BF138707FDA54663E6E604014765
:100FF000A546294539A03307A70285043E97130764
:1010000007FD83870400138607FDE3F6C6FE03860B
:1010100004009306E002FD57631FD6048387140083
:10102000254693861400138507FD6365A60A81474C
:10103000254529433DA09306A0027D57E399D7FC9F
:101040009841930426009105E35307FC3307E040E1
:10105000136808016DBFB38767028506B29793874F
:1010600007FD03860600930806FDE37615FF63D3AC
:1010700007008147B6848386040013068006014575
:1010800093F8B6FF6395C80013F5F60F8504038641
:101090000400930690066303D60663C5C60693064E
:1010A00080056304D61C63C3C6049307500263081B
:1010B000F61A63757401930750021CA0838704001D
:1010C000130514006387071A637375011CB01305B9
:1010D00024005DB51306A0026397C7009C41938668
:1010E0002400910569B7B684814771B7930630062D
:1010F0006303D60893064006E31DD6FA136828005A
:10110000A94699A0930630076304D60C63C5C602AE
:101110009306F0066301D61693060007E31BD6F884
:10112000FD566315D700136818002147938C4500BE
:10113000C14690411DA893065007E303D6FC9308CF
:101140008007C146E31716F71306C006938C4500C7
:10115000E301C5FE13068006E31DC5FC90419375AF
:101160002800639C051033763601DE852285EFF07A
:101170001FA4E68511B51378080163150802BA8724
:101180009306000229A06373740114A00504FD17DF
:10119000E34BF0FE9307F7FF6343E0000547338717
:1011A000E74005079387450063747401944114A0D8
:1011B00013051400229713060002B306A7406344E8
:1011C000D000BE8555BB6373750110A10505F5B749
:1011D00083AC0500138D450063930C00D28C6685AB
:1011E0003EC63AC442C22D3BB247AA8612482247A5
:1011F0006355F00063D3A700BE8613780801631E11
:101200000800BA871306000231A06373740110A0AE
:101210000504BA877D17E3CAF6FE814763C1D7028A
:10122000B68763D3060081473305F4002A97130677
:101230000002B307A74063CFF600EA8535BB33064B
:10124000F40063777601B385FC00838505000CA26A
:101250008507E9B76373750110A10505D9BF6373ED
:10126000740110A01305140001BB13680804C146E3
:10127000E1BDFD1411B3A146C1BD42064186F5B5DD
:10128000A38F0BFE31B303A5C1818280EFF26F9172
:1012900003A9C181EFF0EFAE11CD1384C181AA84FF
:1012A000084019C1EFF06FBD930530042685EFF0BB
:1012B0002FB504C04A856FF00F918280397126CA1C
:1012C0002ED232D436D62A8654109305F0071385D1
:1012D00001B83EDA36C606CE22CC3AD842DC46DE2B
:1012E0008939AA8603A5C18109E9138501B8F137B7
:1012F000F2406244D244216182802686262D1384E6
:10130000C18193E704043EAD9307F00763F4D7006F
:101310009306F007138601B88145EFF06FBB1C40C0
:10132000A6AFF9B7EFF2EF87376500001305850424
:1013300071373765000013054505493737670000E9
:1013400037650000130787078D4605468D45130551
:101350004508AD37376500001305450A85376FF03E
:101360008F8631C599661377F50F938646F309C7C3
:10137000BA96882205058280C167938707F0E98FB6
:1013800081CB21851377F50F3697082325058280B9
:10139000B707FF00E98F81CB41859377F50FB697AB
:1013A0008823450582806181369508216505828004
:1013B00003A741825C41BA976305F502B62395E223
:1013C00083A60182638FF600938681829042631325
:1013D000F60088C2D44354C1DC43B306E540BA9753
:1013E00094C71045B307C700630FF500B62381EE1D
:1013F000938681828C426393A5009CC25441D4C3DE
:101400005C413E9710C78280EFE2BFF983A501835C
:10141000376500001305C50E553583A5C1833765B3
:10142000000013050510593D83A5C18237650000F2
:101430001305451161356FE01FF9EFE29FF613F7D1
:10144000C5FFE1462E8663F1E60693073500F19B62
:10145000930687FE63EAF6041D8F130687FE23A812
:10146000C1828966511713844182938606EAD8C3E4
:1014700094C323A407001CC0BA9723A0F182C966B5
:10148000938606EAB765000094C3D8C398C781461F
:1014900005469385C51A138501C0EFF04FBA184071
:1014A00023A4E1826FE03FF2AA85376500001305AF
:1014B000451B2935C5BFEFE2DFEE39C503A7018320
:1014C0001304350071981389018381446366870E84
:1014D000B1476373F4003144FD55138501C0EFF04B
:1014E0008FB883A7818283A541828328090026853E
:1014F0003386B740B3868840138881826368D600FC
:10150000138501C0EFF02FBE81447DA0B384C500D8
:10151000BA2003AE440061E73307CE40930F47FF84
:1015200063EF8F0A138FC183938EC18213038401EB
:1015300083260F0083A30E001389C1839382C18287
:1015400063EF6F061307C4003297896E3383E5009B
:10155000938E0EEA2322C3012324C3002320D30148
:101560000546D8C0B2A003264300B10863041601A3
:101570002E9618C61387C60022972320E90063F42D
:10158000E30023A0E2000967130707EA9AA0639A21
:10159000970083A601820147B22305EE19C32320D9
:1015A000F800138501C0EFF00FB483A78183B10465
:1015B00081C7A2852685829726856FE0DFE00546F4
:1015C0003697B2A02320EF00E3FFE3FA23A0EE005A
:1015D0005DBFE385D7FCDC430547AE9775BF7286D8
:1015E00031BFEFE21FDC3306B5024111328532C64E
:1015F000D9352A8409C532468145EFF0EFF42285BA
:1016000041016FE05FDC45C5EFE21FD883A741834E
:101610002A8491C3829783A741821389418263669A
:10162000F40883A701826372F408FD55138501C095
:10163000EFF06FA3835764FF930944FF81CB0357F7
:1016400044FF8967938707EA6301F7023765000063
:1016500013050516A531835644FF035664FF37650D
:101660000000CE851305C51791398967938707EA6E
:10167000231AF4FE938781829843231B04FE63F4AC
:10168000E90023A037011387C1831C43832684FF0D
:101690004E85958F83260900B386D940B6971CC323
:1016A000013B138501C0EFF00FA46FE03FD18280B2
:1016B000B70700209386070001479387070021465C
:1016C0008C426396A500131547003E95828005075E
:1016D000C106E317C7FE01458280EFE2FFCA2A84F4
:1016E0002E85AE89328AE9372A89A92C83244900BC
:1016F000930749006390F4048D2493E909F82304C7
:1017000034012146D2852285EFF02FFC83A7018486
:1017100099C322858297EF00007803274900930739
:10172000C4005CC358C42322F90004C8EF006077EA
:101730006FE0DFC884407DBFEFE2BFC683A741846E
:101740002A8491C3829723040400EF00C074544498
:1017500018489307C400D8C214C31CC85CC4EF0067
:1017600040746FE05FC6EFE23FC22E89AA898937D5
:10177000AA84484589332A841DCDD0448145EFF0A1
:10178000AFDC214623043401A3040400CA8522856A
:10179000EFF0AFF383A7018499C322858297EF000E
:1017A000806FD8409307C40091045CC358C49CC0A8
:1017B00004C8EF00006F22856FE05FC0EFE27FBEDC
:1017C00083A741842A8491C3829723040400EF00F5
:1017D000806C544418489307C400D8C214C31CC872
:1017E0005CC4EF00006C2285393D6FE0DFBD03056E
:1017F00085007D81828023900186938701C21387B3
:101800000708DCC39CC3A107E39DE7FE3D47238A8D
:10181000E18423AC018423A6018693874186DCC33F
:101820009CC38280EFE2FFB703A5C186EFF07FB3D0
:101830007D1593173500138501C23E9508411307A6
:10184000C5FE210523ACE184EFE09F976FE0BFB7B1
:10185000EFE23FB5EF002064839701862A89B1E764
:1018600003A5C186EFF0FFAF7D15131735009387F1
:1018700001C2BA9784439387818580439385C4FED0
:101880006305B4028CC383A7C185238AA18499C34D
:101890002285829783C741811305C4019385840003
:1018A00093F7F70F81EBEFE07F934A85EF00605FDE
:1018B0006FE07FB1EF00405FCDBFEFE29FAE2A84C3
:1018C000EF00605D8347440393064401C19B93E7A7
:1018D0001700230AF40283475403139737009387B2
:1018E00001C2BA97D84314C318CCD4C35CC8938739
:1018F000C1869443185C558F98C3EF00805A6FE0FF
:101900009FACEFE21FAA2A847923184C544893070E
:101910004401D8C214C35CC81CCC8347540313973A
:101920003700938701C2BA979843631AF700138769
:10193000C1861C5C144393C7F7FFF58F1CC3952326
:101940006FE07FA8EFE2FFA5B923938701869A2372
:1019500005079AA3B9236FE01FA7EFE29FA4252BE9
:10196000138701861E23FD17C207C1871EA3634B81
:10197000F00023100700352383A7818591C3C93D5B
:101980006FE07FA4392BEDBFEFE2BFA103A48185F7
:101990001923AA842285B5379147230AF402130537
:1019A000C404112E2285A1358547631CF5003C5CDB
:1019B00089EB2285EFF05FD82685E521513D6FE068
:1019C0009FA083A641861307440123A2E186D8C2C3
:1019D0009387418654C81CCCC5B7EFE29F9C2A84EC
:1019E0005105411108CC48C80CD050D014D43A86C7
:1019F00058D49305300236853EC642C4EFF0CFB4CA
:101A0000585410544C5008507117B72600003A969D
:101A1000938686983D21B24722483726000048CC5D
:101A2000230BF402A30AF402232C0402814723228D
:101A300004052324040523280402230A0402232C7A
:101A40000406232E04060147A286130686A6A28555
:101A50001305C404252483A7018799C3228582978F
:101A6000014541016FE03F96EFE2BF935049144DAD
:101A7000795718D954C21307450190C218CD58C9D7
:101A80002D3DEFF0FFDC6FE01F94EFE29F914111DD
:101A9000B2842E8685452A84368946C03AC63EC41D
:101AA00042C2EFF09FC3024892472247B2464A869D
:101AB000A68522851D3741016FE0FF9003A5818532
:101AC0008280EFE27F8C41112E89AA85054532C6BE
:101AD000B684BA893E8AEFF01FC92A8411C92685C7
:101AE000EFF07F9D324609E92285EFF03FCD0144BA
:101AF000228541016FE09F8CAA865288CE87268777
:101B0000CA852285D93DEDB7EFE2BF89692683A753
:101B100081850546AA8603C747033D8B631CC70220
:101B2000D04B984F6308E60258C210C303C6570350
:101B3000938647010E06138701C294CF3297504314
:101B400014C290CF54C3D8CBA92EEFF07FD001455B
:101B50006FE07F873685B126DDBF834745030547A4
:101B6000BD8B639FE702EFE2DF832A842D26834744
:101B70004403AA842285C19B93E72700230AF40229
:101B8000EFF03FD81305C404F1222685192E83A750
:101B90008187014581C72285829701456FE0BF8219
:101BA0007D558280EFE2EFFF41112AC6ED2403A4A8
:101BB00081852A89228555379304C40470008145A4
:101BC0002685D122268539224A85E12CEFF05FC88F
:101BD0001858F9576314F7002328040201454101FE
:101BE0006FE06FFEEFE2EFFBEFE01F8C653F6FE011
:101BF0008FFD834745030947BD8B6390E704EFE200
:101C00004FFA2A84492C5448184C93074401AA845B
:101C1000D8C214C31CCC5CC81305C404252A26856D
:101C200049242285EFF07FC983A74187014581C7F9
:101C30002285829701456FE00FF97D558280EFE2A2
:101C40004FF68346650305473317D70018DD09476C
:101C5000A30AD502230AE502693F83A7818599C3B8
:101C6000EFF01FBF01456FE00FF65449184D930781
:101C70004501D8C214C31CCD5CC98280EFE26FF26B
:101C80004111B2842E86A9452A8436C63AC43EC282
:101C9000EFF0BFA49247B2462247F99B1CB49307CA
:101CA000440144CC14D02324040258D01CCC5CC87A
:101CB00041016FE04FF1EFE2CFEE2A84E92AAA84D6
:101CC000228565372685F12A2285EFF0FFA601459A
:101CD0006FE06FEFEFE2EFEC2A84752AAA84228589
:101CE00069371C342685F99B1CB4652A83A7C184F7
:101CF00099C322858297EFE04FF85C503E9508D457
:101D0000592A138781880328470037060080938764
:101D100081881346E6FF98436315F8029386C187CE
:101D20009042050690C29306440154C358C894C318
:101D30001CCC1C3493E717001CB4A52201456FE0AE
:101D40008FE8544B0C546385B6008D8EE378D6FC37
:101D5000BA87D1B71C35858B8DC7EFE28FE483A797
:101D600081842A8491C382973D22AA842285EFF040
:101D7000DFEF26853D221C340145F99B1CB46FE042
:101D80008FE47D55828085476381F50263C5B70086
:101D900085C1014582808947638FF5008D47E39AAD
:101DA000F5FE1C3593E7270009A85C511CC2D5B786
:101DB0001C425CD1F9BF1C35F59B1CB5D9BFEFE2C5
:101DC000CFDBEFE08FEB2A8CF920B70900802A8A5D
:101DD0009384818893C9E9FF8D4B804063169400FA
:101DE0005285C1206FE0EFDC48481309C4FE33057B
:101DF000AC40E3E7A9FE83A7018899C34A8582978F
:101E00004A85EFF09FE61C4448448297EFE0EFE6F6
:101E100083A741882A8C99C34A858297834754FFB8
:101E200013F7E70FA30AE4FE8D8BE39877FB4A854F
:101E3000EFF05FEA5DB793878188DCC39CC3828043
:101E400082801106719A2A8837C7ADDE130506F81D
:101E5000AA871307F7EE631EF600A167938707882A
:101E60002322D6F82324B6FA232006F92324F6F8F1
:101E7000828098C39107C5B737F700E01C43B706C7
:101E80000080D58F1CC3828037F700E01C43860793
:101E900085831CC382802165130505807315053079
:101EA0008280731005308280EFE2AFCF1387818983
:101EB00018439387818919E323A8A18823AAB188AD
:101EC000054798C3553F6FE00FD02A8781471843D5
:101ED0006314A7003E8582808507D5BFB707EFBE94
:101EE00037E700E0938707083CC701458280EFE2AF
:101EF0004FCB376500001305051FEFF02FBC0145E0
:101F00006FE06FCCEFE2EFC92A84FD54377900000F
:101F10007D14631494006FE00FCB13058995EFF0E7
:101F2000EFB9FDB7EFE24FC60041AA843779000050
:101F3000B7790000631494006FE04FC89305C4FEA6
:101F40001305C995EFF08FB71C4063869700138582
:101F50000996EFF0AFB60040F1BFEFE28FC42E89D3
:101F6000EFE01FFC2A84EFF0FF9D83240900639CAF
:101F70002401EFF09F9EA14763C3870011E0214435
:101F800022856FE04FC4138544FFEFE07FF9635370
:101F9000A4002A848440E1BFEFE22FBE0545EFF0A4
:101FA0002FF1B7690000130945002A84CA851385FB
:101FB000494AEFF09FFAAA85AA8437650000138684
:101FC000494A1305C54AEFF06FAF2685EFF09FF33E
:101FD000376500001305054FEFF04FAE4040B7697D
:101FE0000000054A894A376B0000B76B0000376C68
:101FF0000000B76C0000376D0000631589000145D3
:102000006FE02FBB0347940213850953930644FFE7
:102010002146A685EFF08FAA834784021385CC530F
:10202000BD8B638E470113058C54638A570113855A
:102030004B5591C711476396E70013050B56EFF018
:10204000EFA74C4C93073002AE8698226306F70246
:102050001050930740060848B295B386D540B38622
:10206000F602585C5C50898D1305CD56B3D6C60276
:10207000EFF0CFA4004051B78506C1BFEFE2CFB06B
:1020800041110945EFF0CFE293094500376900009F
:102090002A84CE8513054944EFF03FECAA85AA8433
:1020A000376500001306494413050545EFF00FA1FD
:1020B0002685EFF03FE5376500001305C546EFF0D4
:1020C000EF9F4040376A0000B76A0000377B00008E
:1020D00063968900014541016FE04FAE1A281C4408
:1020E000930644FF1309840036C63AC44A85630642
:1020F000F902EFF09FDD2247B246AA872146A68566
:1021000013854A48EFF08F9B4A85EFF0BFE1130536
:102110008B57EFF0AF9A004065BFEFF01FDB22470F
:10212000B246AA872146A68513054A49EFF00F99C2
:10213000DDB7EFE26FA541111145EFF06FD79309BD
:102140004500376900002A84CE8513058928EFF001
:10215000DFE0AA85AA8437650000130689281305E5
:102160000529EFF0AF952685EFF0DFD93765000040
:102170001305452BEFF08F944040376A0000B76A93
:102180000000377B000063968900014541016FE044
:10219000EFA21C4413098400930644FF1848630906
:1021A000F9024A8536C63AC4EFF03FD22247B2461A
:1021B000AA872146A68513854A2DEFF02F904A85E0
:1021C000EFF05FD613058B57EFF04F8F004065BFE0
:1021D0002146A6851305CA2EEFF04F8EC5BFEFE24C
:1021E000AF9A41110D45EFF0AFCCB769000013096C
:1021F00045002A84CA851385093EEFF01FD6AA85BB
:10220000AA84376500001386093E1305853EEFF06A
:10221000EF8A2685EFF01FCF376500001305C54014
:10222000EFF0CF894040B76900006316890001458F
:1022300041016FE0AF98930644FF1305840036C652
:10224000EFF0BFC8034834015C48B246AA88214772
:102250002146A6851385C942EFF04F860040F1B7AD
:10226000EFE28F9241111545EFF08FC493094500BD
:10227000376900002A84CE8513050930EFF0FFCDC1
:10228000AA85AA8437650000130609301305853036
:10229000EFF0CF822685EFF0FFC63765000013050B
:1022A000C532EFF0AF814040376A0000B76A0000E6
:1022B000377B000063968900014541016FE00F9074
:1022C0007A285E281044930644FF1309840036C61A
:1022D0003AC43EC24A856307C902EFF01FBF924766
:1022E0002247B2462A882146A68513858A34EFE024
:1022F000FFFC4A85EFF01FC313058B57EFE01FFC6F
:1023000000404DBFEFF07FBC92472247B2462A887B
:102310002146A68513050A36EFE05FFAD5B7EFE24E
:10232000AF8641111945EFF0AFB893094500376901
:1023300000002A84CE8513058937EFF01FC2AA85D5
:10234000AA84376500001306893713054538EFE086
:10235000FFF62685EFF01FBB376500001305053A31
:10236000EFE0DFF54040376A0000B76A0000377BD6
:10237000000063968900014541016FE02F841A2C0B
:102380001C44930644FF1309840036C63AC44A85A8
:102390006306F902EFF07FB32247B246AA872146CF
:1023A000A68513858A3BEFE07FF14A85EFF09FB762
:1023B00013058B57EFE09FF0004065BFEFF0FFB0D3
:1023C0002247B246AA872146A6851305CA3CEFE0FC
:1023D000FFEEDDB7EFD25FFB5D712545EFF04FAD4E
:1023E0009965130600052A84130945009385C5E9FC
:1023F0000A85EF301019B7690000CA8513850922D4
:10240000EFF0BFB5AA85AA843765000013860922BC
:1024100013058522EFE09FEA2685EFF0BFAE376512
:10242000000013050525EFE07FE94040D149376AF8
:10243000000063168900014561616FD03FF81C44BC
:10244000930644FF63E0F90298088A07BA9703A746
:1024500007FB1C282146A68513054A27EFE01FE647
:102460000040C1BF4647F5B7EFD21FF22945EFF054
:102470002FA4B7690000130945002A84CA85138573
:102480004959EFF09FADAA85AA84376500001386ED
:1024900049591305C559EFE07FE22685EFF09FA665
:1024A000376500001305455CEFE05FE14040B76928
:1024B0000000376A0000B76A0000631E8900EFD091
:1024C000DFFBAA85376500001305C561EFE01FDF5C
:1024D00001456FD0BFEE5C4C184C1385895E9306A6
:1024E00044FF2146A685EFE07FDD8347D4FF1385B7
:1024F0000A60858B99E31305CA60EFE03FDC00407A
:102500006DBFEFD27FE8376500001305851FEFE050
:10251000FFDA03A4018AB7690000376A000083A7C5
:10252000418A6365F40001456FD05FE904400946C4
:102530009385C9202685EF30F01319C55040A68534
:1025400013050A21EFE09FD73104D1BFEFD2DFE3BB
:10255000377500001305C5ABEFE05FD603A4018A11
:10256000B7790000377A000083A7418A636BF400D3
:102570003775000013058557EFE05FD401456FD034
:10258000FFE304401946938589AD2685EF30900E10
:1025900001E950409385640013050AAEEFE01FD2B5
:1025A0003104D9B705458280EFD21FDE79712A84C4
:1025B000AA9593060002254783070400B38485404B
:1025C0006385D70A6383E70A0145638B04100149D9
:1025D00013070002A546B307240183870700638A17
:1025E000E7086388D7086314990883A9018A83AA36
:1025F000418A377B000063F0590903AA0900194694
:1026000093058BAD5285EF30F00659E54A86A285D9
:1026100013056A00EF30100641E14A9A83076A0009
:10262000A5EF83A989006388090413068002814508
:102630002800EFD01FDA13098100CA86A28701455E
:10264000014713080002A548294313062002130E70
:10265000C005838507006384050163961505631F24
:102660009702A9476303F50469A80504B1B70509F2
:102670009DB7E31C09F6A287038707001377F7FDD0
:1026800079E737750000130545AA23800700A28566
:10269000EFE0DFC27D55A9A0B109B1BF23800700DB
:1026A000050785077DB763106504377500001305BE
:1026B00005A8EFE0BFC00018B7740000832509002B
:1026C000138504AA1109EFE07FBFE31989FE37756E
:1026D000000013058557EFE07FBE29452C00829945
:1026E00045616FD0BFCD637E970005056392C50439
:1026F000850705079CC2838507006381C502636463
:10270000970069FD8DBF838E17006396C5016394A2
:10271000CE008507050785070507F1BFE37397FE20
:1027200023800700050785079106E36497F2D1BF70
:102730009CC2838507006389050163871501E30255
:1027400097FC85070507F5B7E36097FE5DBF850732
:1027500025B7EFD29FC28307050099E78145014560
:10276000EFF0DFDE6FD0FFC403AA018AAA8981449B
:102770000149377B0000B77B000083A7418A63696A
:10278000FA00EDD04A86A6854E85EFE00FF4D9BF5A
:1027900003240A00194693058BAD2285EF30806D26
:1027A00021E14E85EF30E06B19042A86A2854E8523
:1027B000EF30406C15E5631709002285EF30606A41
:1027C0002A89A284A68722870386070001EE858FC7
:1027D00063D327013E89A28513858BAEEFE01FAE40
:1027E000310A61BF83060700FDD2E312D6FE8507DA
:1027F0000507D9BFEFD2FFBAEFF00FFA01456FD04E
:102800009FBCEFD21FBAEFE03FC001456FD0BFBB06
:10281000EFD23FB903A5C189EFE0EF8C01456FD03E
:102820009FBAEFD21FB8B77700009387475823A00D
:10283000F18AB77700009387476D23A2F18AB777B3
:1028400000009387476D23A4F18AB7770000938730
:10285000476D93050021054523A6F18A1384C1899C
:10286000EFE03FD808C019E9377500001305C5B976
:10287000EFE0DFA47D5422856FD0FFB4B7350000B0
:1028800037750000A9472D47930600400146938500
:10289000259A130545BBEFF0CFA2AA840840B7756F
:1028A0000000814601469385C5BBEFD05FF9014426
:1028B000F9D02685EFF0AFB87DBFEFD29FAEEFF035
:1028C0007FCE0DC5B7750000938585B6138501CA07
:1028D000EF302058B7750000938585B7138501CA7E
:1028E000EF304055138501CA6FD0FFADB7750000BA
:1028F000938505B7E1BFEFD2DFAA2A8437750000C0
:10290000130585BDEFE09F9BEFF03FFBAA85377570
:1029100000001306A41B130505BEEFE03F9A014516
:102920006FD07FAAEFD2FFA741112AC6EFD07FC593
:10293000B24511E9377500001305C5B7EFE01F98E0
:1029400041016FD05FA883A7C189AA841384C1897C
:1029500083A7C720E386A7FE93053014EFD05FCA94
:1029600065F11C4003A5C72009C9EFD01FD11C4049
:10297000814503A5C720EFD09FD70040130600056F
:1029800081451305A41BEFD0DFA4B7350000231544
:10299000042023269420938505812685EFD03FD5FA
:1029A00045B7EFD21F9D83A7C18941119384C18987
:1029B00003C74702136717002382E70283A7C720D4
:1029C00091E7EFE05F8C19C1EFF0DFF5EFF0FFEE7C
:1029D000EFE0DF8E377B0000B77B0000B7790000A7
:1029E000377A0000B77A0000377C0000B77C00001F
:1029F0009C4085461306F10003A5C720FD55EFD086
:102A00005FCB8547631AF5000309F100ED4780406D
:102A10006319F90008D0E9BF8840FD55EFD0BFE445
:102A2000C1BF1C506392A7029307B0056315F9005C
:102A300089471CD075BF23200402E30B09FAA54780
:102A40006314F9120149D1A80947E398E7FE23204E
:102A50000402930710046312F9046E30D1D9FD15F6
:102A6000C205C1816EB09307A41B13070005B3858F
:102A7000E502130600053E859385A502A295EF3079
:102A80004030EF30003E1375F50F2305A420A30559
:102A9000A4202285EFF03FE6A1BF93072004631135
:102AA000F90216347E301387F6FF63D8E7008507F6
:102AB0007EB09307A41B6E304DBF9DDA7AB0D5BFB0
:102AC000930740046310F9028347B42095D313851C
:102AD00049BCEFE0AFFE98408347B720FD17A30540
:102AE000F72039B793073004E319F9F48347B4208A
:102AF0000347A420E3FEE7EE3E948305A41B138561
:102B00008ABCEFE0AFFB98408347B7208507C1BF81
:102B1000138549BCEFE08FFA050980408347B42054
:102B2000E348F9FE13058A57EFE04FF9EFF09FA74E
:102B300085471304A41B6315F5002285EFF07FC1C0
:102B4000EFF0BFD72286AA8513850CBEEFE00FF702
:102B500080401305A41BEF30C0301375F50F23051B
:102B6000A420A305A42069B59307F0076305F90025
:102B7000A1476315F9088347B420E38B07E60346B2
:102B8000A420FD1793F7F70F7D161376F60F230594
:102B9000C420A305F42063F8C7049385B71B1385ED
:102BA000A71B1D8EA2952295EFE0AFAD9C4013852B
:102BB000CBBC03C7A7203E97230D071A83C5B720B8
:102BC0009385A51BBE95EFE06FEF9C4003C4B72033
:102BD0009C4083C7A720E3CD87E0138549BCEFE085
:102BE000EFED0504F5B713054BBDEFE02FED9C406D
:102BF00003C7A720BA97238D071ADDBB3547834744
:102C0000A4206305E9002947631EE90EB9CB0359E7
:102C100084029147130DA41B63FB2709930DA4168F
:102C200013060005EA856E85EF3060131DC9130990
:102C3000A4024A851309090513060005CA85EF3069
:102C40004014E3982DFF1306000581456E85EFD0F3
:102C50004FF80346A420EA856E85EF308012954731
:102C60001EB41E347EB0EFF0FF9385476312F50269
:102C70009C4083C74702858B89C713058A57EFE0BD
:102C8000EFE388408345A5201305A51BEFF0DF91F6
:102C9000EFF0BFC2EFE08FE28040130600058145F0
:102CA0001305A41BEFD0EFF22315042091B36301A9
:102CB00009021305F9FF930700053305F502130612
:102CC0000005EA851305A5022295EF30400951D988
:102CD000930D00053305B90313060005814513055F
:102CE000A5022295EFD0EFEE0A340346A420EA8530
:102CF0003305B5031305A5022295EF3080081E3475
:102D00008507B9BF1307F0046374F7002305042097
:102D10000346B4208347A4206370F6089305A61BDE
:102D20001305B61BA2953386C7402295EFE06F9539
:102D30008C4083C7B5203387F500230D271B03C7BD
:102D40004502058B01CB9387A71BBE951305CC9538
:102D5000EFE0CFD69C4003C4B7209C4083C7A72098
:102D60006346F40298408347A7208346B72085072F
:102D7000850693F7F70FA305D7202305F7209306C1
:102D8000F004E3F7F6C6231507209DB1138549BC6F
:102D9000EFE0CFD20504D1B7A297238D271B83473D
:102DA0004402858BE1D3CA8513858ABCEFE00FD13D
:102DB00055BF7C4123280504232A05049C4381CB6D
:102DC000EFD22FDE9305850482976FD0CFDF0145C8
:102DD0008280EFD26FDB36899DCAAA843284B30920
:102DE000D600294A1C20639B4701BE2C93F7070499
:102DF00091C7FC40B54526859C478297FC408305DA
:102E0000040026859C4705048297E31D34FD4A850E
:102E10006FD0CFDAEFD2EFD893F705102A8491C79D
:102E20001A2D61551377071035CF13F7054011C7D9
:102E30001A2C61551377074035C713F7050493041F
:102E4000000401E7262C93F40404384893F5F50FA9
:102E50002EAC39EBA1C76844298142054181310577
:102E6000EFE06FE570442A893105298242064182EC
:102E700081452320A900EFD03FED232209003E2CFD
:102E8000232409002328240593E707103EAC7C4047
:102E900013060010C145DC43228582973E2C014574
:102EA000DD8C26AC6FD02FD2F5DB93E505102EAC70
:102EB000F5B70948AA8763810503EFD28FCE0D4885
:102EC0006382050305476399E5041A2D1377F7FD1F
:102ED0001AAD01456FD02FCF1A2D136707021AAD17
:102EE00001458280328775D6504274454C2D298227
:102EF000A9824206C2064182C1826304D6001D45F2
:102F0000F1F91443B4C75443F4C7E1D5F443BA8587
:102F10003E859442829675BF7C41DC4382975DBFBB
:102F2000EFD28FC63684B1CA3E2DAA89328993F773
:102F30000710B6849DE37D5AA94A83A749044E85AC
:102F4000DC478297630945012300A900FD140509A8
:102F500063035501FDF0058C0DA02449368A854A8E
:102F6000EFE07FF3FE20DA202A869444631AF7000C
:102F700081EAEFE01FF33304444122856FD00FC490
:102F800098403E97034B070003A7C9048507C20773
:102F90002983C1834207FEA0418363E4E7002393B2
:102FA00004006394560123A404003285EFE07FEF10
:102FB0007D1A230069010509E3140AFA6DBF582D33
:102FC000854763ECE7023E2D93F707109DC7EFD2CC
:102FD0004FBD2A842849EFE00FE33E2C2328040448
:102FE0001306001093F7F7EF3EAC7C40C5452285F1
:102FF000DC43829701456FD00FBD01458280EFD23F
:103000004FBA37370000130727DB18D537370000D2
:10301000130747E158D5373700001307E7FB18D9E6
:1030200037370000130707F258D937370000130766
:1030300027DD18DD37370000130727EB420658DD80
:1030400034C14182232A05002320050223220502E0
:10305000EFD0CFD76FD02FB793F5F50F854763919A
:10306000F50AEFD26FB220494111AA847D598549F2
:10307000FC402685DC4782972A8A63072505EFE016
:103080009FE15A201C40BA97238047015E20F844F4
:103090008507C2072983C18342075EA0418363E499
:1030A000E7002312040076205E20639CD70085078A
:1030B000C207C1837EA02324340163E4E700231305
:1030C0000400EFE01FDE6DB79C5085C3EFE0BFDC6E
:1030D0005A206E20636EB700B305B7402EC6EFE0EE
:1030E0005FDC9C50B2452685829741016FD00FADC1
:1030F000FC44998DA983C207C183B385B740F9BF4A
:10310000828001CEEFD2EFA97841B2878E23184397
:103110003222029701456FD00FAB7D558280EFD2EE
:103120004FA8138741D278432E86AA85184313856A
:1031300041D202976FD02FA9EFD2AFA6138741D209
:1031400078432E86AA855843138541D202976FD0C3
:103150008FA7EFD20FA5138741D27843AA85138595
:1031600041D2184702976FD00FA605C61147639248
:10317000E602EFD20FA37C410E2241119C4736C6D6
:1031800032C482972246B2462AA2368541016FD0C8
:103190008FA38146368582801DC2B2871146639017
:1031A000C602EFD20FA07841B2238E2358434111BB
:1031B00036C60297B246410136856FD0CFA0814610
:1031C00036858280EFD2EF9D938741D24947D8CB95
:1031D000373700001307A716D8DB3737000013076F
:1031E000871998DF3737000013072710ECC3B0C3E7
:1031F000AA850D46138541D223A0070223A2070208
:1032000023A4070223A6070223A80702D8DFEFD0D2
:10321000EFBB01456FD02F9BEFD2AF98B7070020CF
:1032200003A7072A9307803EC1563357F702B7E733
:1032300000E02386D7402387D740856623A0D71098
:10324000916623A0D710B7F700E023A0070023A2C0
:103250000700014690C78146D4C781461306F7FF91
:1032600090CBD4CB3D4798C3EFD08FA7B7050120B3
:103270001385C122EFE06F9C37750000130585C5EB
:10328000EFE0CF806FD02F9473110134EFD01F8CFB
:10329000B7F700E023A20700EFD08F9EEFD0FF8D9D
:1032A0007311013473002030232605000CC150C176
:1032B00023240500054582805C4554411845850757
:1032C000B3E7D702638EE70058451C41BA978CA339
:1032D0005C4558418507B3E7E7025CC50545828038
:1032E0007955828018455C45630FF70018451C41ED
:1032F000BA979C239CA11C4558418507B3E7E70278
:103300001CC505458280014582805C4518454841C1
:10331000998FAA9733E5A7028280814785461307D4
:1033200000023396F6006306A6008507E39BE7FEDE
:10333000FD573E858280EFD2CF868545130500027A
:10334000EF1030736FD02F88EFD2AF8585452145C0
:10335000EF1030726FD02F87EFD2AF8485451145C3
:10336000EF1030716FD02F86EFD2AF838545414586
:10337000EF1030706FD02F85EFD2AF8285451305E7
:103380000004EF10106F6FD00F84EFD28F819D6516
:10339000377500000146938505C613058534EFF0A7
:1033A0007FE26FD04F829307400663ECA70093172C
:1033B00045001D65130585CF3E951841FD576313E4
:1033C000F70001458280EFC2DFFD411113F5F50FD3
:1033D00032C6EFF05FFD11C54E2532460845EF10AD
:1033E000B04941016FC03FFEEFC2BFFB13F5F50FBF
:1033F000EFF07FFBAA87014589C7CE278847EF10EA
:1034000010476FC05FFCEFC2DFF9011113F5F50F34
:103410003284EFF05FF905C55C412AC682973245D8
:103420005C45FC82C1473ECE8D473ECC09C4154762
:10343000631AE40002CE08454C08EF1050370561CE
:103440006FC07FF805476315E40091473ECEE5B7AE
:103450006315F40093078002D5BF89476315F40014
:1034600093078004E5B791476314F400D147F9BF8F
:1034700099476314F400F147D1BF9D47E31DF4FA67
:10348000E147E9B7EFC25FF013F5F50FAE84B289FB
:10349000368A3A89EFF03FF1994731CD4845EFF050
:1034A000DFE73D472A8499476367A704EFE0BF9EA3
:1034B000B146B306D402B7070020138707082A864F
:1034C00093870708369783160700639F96004C433F
:1034D000639C45012E236399350118476316270124
:1034E000EFE03F9C814701A87D576389E600328564
:1034F000EFE03F9B9D473E856FC05FEC3145330554
:10350000A4023E9506A1232245012311350123245F
:1035100025013285F1B7EFC2DFE813F5F50FEFF0C3
:103520009FE819471DC94845EFF03FDFBD472A8492
:10353000194763E4A702EFE01F96B1473304F40292
:10354000B7070020938707087D57A2978396070047
:103550006398E600EFE0FF9401473A856FC0BFE64D
:1035600041677D1798C323A2070023A40700DDB796
:10357000EFC29FE1011113F5F50F328AEFF0BFE2C0
:10358000994721C185442A8463159A104845EFF074
:10359000DFD83D47AA8499476365A702EFE0BF8F54
:1035A000B14AB38754033709002013090908AA89CF
:1035B0003E9903170900FD576319F700EFE07F8E6E
:1035C00099473E8505616FC07FDF5C4082978545E6
:1035D0000545EF10104A5C440D473AC47C823EC852
:1035E0008357290002CA52CE638C4709C1C70947D5
:1035F000638DE70808444C00EF10701B1844B717A0
:103600000140938607C005456302D7020945630F51
:10361000F700938707400D45630AF700B72701407D
:103620009387078001456313F700114593F5F40F65
:10363000EF1030250808EF10700E9D67938787C73D
:103640008E04BE94D04037E700E093060005B30730
:10365000C7002380D74093575600938707048546B9
:103660008A07B396C600BA9794C34E85EFE07F836E
:10367000814781BF930780023EC6A1473ECC9DBFD4
:10368000930780043EC656CCB5B791473EC6C147A6
:10369000F5B79947E3170AF24845EFF01FC83D47D1
:1036A0009947E360A7F2931735001D65130585C799
:1036B0003E9558419357570093870706B394E4000B
:1036C0008A0737E700E0BA9784C35DB7EFC27FCDC2
:1036D000EFF0BFC4B1473305F502B7070020938769
:1036E00007083E955C4199C3084582976FC0BFCDDE
:1036F00073110134EFD08FC50545EF10D00819C5FF
:103700000545EFF0BFFC0545EF10D009EFD0EFC63F
:10371000731101347300203073110134EFD00FC3E3
:103720000945EF10500619C50945EFF03FFA094564
:10373000EF105007EFD06FC47311013473002030C5
:1037400073110134EFD08FC01145EF10D00319C5AC
:103750001145EFF0BFF71145EF10D004EFD0EFC1E6
:10376000731101347300203073110134EFD00FBE98
:103770002145EF10500119C52145EFF03FF52145D6
:10378000EF105002EFD06FBF73110134730020307F
:1037900073110134EFD08FBB4145EF10C07E19C5C6
:1037A0004145EFF0BFF24145EF10C07FEFD0EFBCD5
:1037B000731101347300203073110134EFD00FB94D
:1037C00013050002EF10207C1DCD13050002EFF061
:1037D000FFEF13050004EFF07FEF13050008EFF093
:1037E000FFEE13050010EFF07FEE13050020EFF061
:1037F000FFED1305003EEF10E07AEFD00FB8731124
:1038000001347300203013050004EF10C07755FD1C
:1038100013050008EF1020774DF913050010EF1085
:10382000807645F513050020EF10E07559FDF1B7DE
:1038300073110134EFD08FB113050040EF10A07465
:1038400029C113050040EFF07FE8056513050580E9
:10385000EFF0DFE70565EFF07FE70965EFF01FE7C1
:103860001165EFF0BFE62165EFF05FE641651305F6
:1038700005C0EF102073EFD04FB073110134730007
:103880002030056513050580EF10E06F5DF90565D3
:10389000EF10606F5DF50965EF10E06E5DF1116589
:1038A000EF10606E59FD2165EF10E06D59F9E1B739
:1038B00001458280EFC2FFAE9C412041A1464111EB
:1038C0001CC0B1473EA4DC412316040013F7F700E7
:1038D0006301D702A546631ED70005675AA013D718
:1038E00047000D8B01C785466308D70023130400EA
:1038F00031A023120400E5B709677AA099838D8B64
:1039000005476389E70081C709476389E7062314F0
:10391000040021A0930700601EA41848B747014087
:10392000938707806318F704116585451105EF102B
:10393000501493070020B71401407C820D49E147E1
:103940004C00138504803EC64AC4EF1040669307BE
:1039500000407C824C009147138504803EC64AC4D7
:10396000EF10E0640848A285EF1070140848854500
:10397000EF10F01C014541016FC0FFA49307004008
:1039800061BFEFC27FA0138441DC930750035CC882
:10399000B74701401386C1D69387078074461CC879
:1039A0009D679387C7347CC2B70700C0F58FC16697
:1039B000A106716713070720D58F1165411138C61D
:1039C0007CC68545B7070C00110518C01CC423220E
:1039D000040023160400EF10D009B7190140930723
:1039E00000207C820D4AE1474C001385098052C4B7
:1039F0003EC6EF10C05B930700407C824C009147AD
:103A0000138509803EC652C4EF10605A084893855A
:103A100041DCEF10D00908488545EF105012B7750A
:103A20000000938641DC13063010938585C513850D
:103A3000C1D6EFF0CFDC014541016FC03F98EFC226
:103A40005F962041930500020848EF10101519C534
:103A50001C48CA231375F50F6FC0FF967D55EDBF47
:103A6000EFC23F9424412E84884893050004EF1050
:103A7000D0127DD99C4842044180C2A305456FC045
:103A80009F94EFC21F92C1473841638BF502C5472F
:103A90006395F502544B054693D756009387070666
:103AA0003316D6008A07B7E600E0B69790C3014602
:103AB000084B93055052EF10F00901456FC0BF90BD
:103AC000544B054693D75600938707043316D60008
:103AD0008A07B7E600E0B69790C30546D1BF41110B
:103AE00022C626C473110134EFD04F869387C1D606
:103AF000A043930550520848EF10D00A19C98545D4
:103B00001385C1D6EFF04FD5084893055052EF10FA
:103B1000300DEFD08F86731101343244A24441013D
:103B20007300203073110134EFD04F8237750000DD
:103B30001305C536EFD08FF8EFD02F847311013401
:103B40007300203073110134EFD04F8037750000BF
:103B500013050536EFD08FF6EFD02F8273110134A5
:103B600073002030EFC2FF83377500001305C5379F
:103B7000EFD0CFF49D22B707002083A5072A377521
:103B8000000013050539EFD06FF3EF108038AA85D8
:103B9000377500001305053AEFD04FF2152801459F
:103BA0006FC07F82EFC2EFFFEF10D005EF10D0069D
:103BB000EF10102D6FC03F81EFC2AFFEEF1020114C
:103BC000EF00907CEF00D076EF0050796FC0AFFF30
:103BD000EFC22FFDEFF01FFDEFF01FFE6FC0AFFE35
:103BE000B71702409843B706FFF04111136717005B
:103BF00098C3D84337060200758FD8C39843B706D9
:103C0000F7FEFD16758F98C39843B706FCFFFD16A7
:103C1000758F98C3D843B70601FFFD16758FD8C3BB
:103C20009843B70600ECFD16758F98C33707FF0061
:103C300098C723A6070202C402C69843C166558FDF
:103C400098C3B716024005679C42F18F3EC6A24753
:103C500085073EC4B24781E7A247E397E7FEB7175F
:103C600002409C431397E7006357070685473EC60B
:103C700032478547631FF704B7170240D843B7069A
:103C8000C1FFFD16D8C3D843D8C3D8431367074034
:103C9000D8C3D843758FD8C3D843B7062900558FEA
:103CA000D8C39843B7060001558F98C3984393161D
:103CB0006700E3DD06FED843B7160240719BD8C308
:103CC000D84313672700D8C32147DC42B18BE39E5A
:103CD000E7FE4101828002C661BFB7160240D842AA
:103CE000B70700201146318B9387072A6305C70069
:103CF00021466308C70237177A001307072098C3C5
:103D000037170240584311839376F7003707002096
:103D1000130707143697142398433357D70098C3D3
:103D20008280D842D442416649833D8BF18E13068E
:103D3000270015CF3D47630FE6024147630FE602B8
:103D4000454781456313E6004146A1E237470240FB
:103D500003270780418B0DC737177A001307072009
:103D60003306C70290C3C9DD9843058349BF814527
:103D70004946E1BF85453546C9BF81453D46F1B756
:103D800037173D0013070790E1BF3715024058551C
:103D90009316F700585563DF060411833D8B930695
:103DA000170037177A00130707203357D70298C335
:103DB0005455A182BD8A8DE295463307D70205830B
:103DC00098C337170240585794433D8B050733D7A4
:103DD000E60298C3984369B705456394A600E54693
:103DE000E9BF3D456396A600D1463387E602C9BFC9
:103DF0008906E5BF3D8B9306170037177A00130736
:103E000007203357D702F1B701A07390123497D12E
:103E1000FF1F938121C917C100201301A11E17455F
:103E200000001305258D97C5FF1F9385A51D1386DB
:103E3000818063FAC5008322050023A05500110587
:103E40009105E3EAC5FE138581809385C1226377DE
:103E5000B500232005001105E36DB5FEFD4273900A
:103E600002BCFD4273904280B782000093820280C0
:103E70007390023097C2FFFF9382021993E23200DF
:103E800073905230EFF0DFD597C2FFFF9382026F3D
:103E90007390123473002030EFC2AFD02A84B28402
:103EA0002E89130640038145138581E7EFC06FD249
:103EB00083A7C18C138741E723AAF1E693875400B7
:103EC0005CB3B70700209387071AB427BC37138663
:103ED00041E774A37CB383A7418B63928704930764
:103EE00060101EA6814763E197082696DD473CA631
:103EF00003A5018B13068003938541E7EFC05FACF8
:103F000019C53775000013058550EFD02FBB3775E5
:103F1000000013058551EFD06FBA6FC0CFCA83A7D9
:103F2000818B639587009307701065BF83A7C18B52
:103F300063958700930720106DB783A7018C639565
:103F400087009307801071BF83A7418C6397870018
:103F50000D4718A6DC4F1CB671B783A7818CE3937D
:103F600087F893074010B5BF3307F90014233307D0
:103F7000F600850734A793F7F70FB5B7EFC26FC206
:103F80002A84B2842E89130640038145138581E774
:103F9000EFC02FC483A7C18C138741E723AAF1E6A2
:103FA000938754005CB3B70700209387071AB427A0
:103FB000BC37138641E774A37CB383A7418B63921C
:103FC0008704930760101EA6814763E19708269631
:103FD000DD473CA603A5018B13068003938541E7CB
:103FE000EFC01F9E19C53775000013058550EFD02F
:103FF000EFAC3775000013058553EFD02FAC6FC0C1
:104000008FBC83A7818B639587009307701065BF72
:1040100083A7C18B63958700930720106DB783A793
:10402000018C639587009307801071BF83A7418C33
:10403000639787000D4718A6DC4F1CB671B783A79E
:10404000818CE39387F893074010B5BF3307F900DD
:1040500014233307F600850734A793F7F70FB5B796
:10406000EFC22FB42A84B2842E89130640038145FF
:10407000138581E7EFC0EFB583A7C18C138741E7B4
:1040800023AAF1E6938754005CB3B7070020938717
:10409000071AB427BC37138641E774A37CB383A700
:1040A000418B639C8702930760101EA6814763EBD8
:1040B00097062696DD473CA603A5018B13068003D1
:1040C000938541E7EFC0DF8F19C5377500001305F1
:1040D0008550EFD0AF9E6FC00FAF83A7818B6395E4
:1040E000870093077010D1B783A7C18B63958700B2
:1040F000930720105DBF83A7018C6395870093070A
:10410000801065B783A7418C639787000D4718A679
:10411000DC4F1CB661BF83A7818CE39987F89307B6
:10412000401061B73307F90014233307F600850701
:1041300034A793F7F70FA5BFEFC2AFA62A84B284C6
:104140002E89130640038145138581E7EFC06FA8D0
:1041500083A7C18C138741E723AAF1E69387540014
:104160005CB3B70700209387071AB427BC371386C0
:1041700041E774A37CB383A7418B639287049307C1
:1041800060101EA6814763E197082696DD473CA68E
:1041900003A5018B13068003938541E7EFC05F827F
:1041A00019C53775000013058550EFD02F9137756D
:1041B00000001305C54EEFD06F906FC0CFA083A74E
:1041C000818B639587009307701065BF83A7C18BB0
:1041D00063958700930720106DB783A7018C6395C3
:1041E00087009307801071BF83A7418C6397870076
:1041F0000D4718A6DC4F1CB671B783A7818CE393DB
:1042000087F893074010B5BF3307F900142333072D
:10421000F600850734A793F7F70FB5B7EFC2CF962F
:104220002E89B284814513068003138541E7EFC0D0
:104230004F9A9387C4FF938941E7A382F90083478C
:1042400029001947938641E7F91793F7F70F636D34
:10425000F7001D678A071307073BBA979C438287BD
:1042600083A7C18B23AAF1E681471386F4FF63EA93
:10427000C70403A5018B13068003938541E7EFC0B4
:104280002FF419C53775000013058550EFD00F8343
:10429000377500001305454AEFD04F826FC00F926B
:1042A00083A7418C23AAF1E683473900DCA26DBFC6
:1042B00083A7818C45BF83A7818B6DB783A7018CB2
:1042C00055B73307F90048233387F600850768A3FD
:1042D00093F7F70F69BFEFC22F8B2E89B284814508
:1042E00013068003138541E7EFC0AF8E9387C4FFA9
:1042F000938941E7A382F9008347290019479386F0
:1043000041E7F91793F7F70F636DF7001D678A0709
:104310001307C73CBA979C43828783A7C18B23AA04
:10432000F1E681471386F4FF63EAC70403A5018B16
:1043300013068003938541E7EFC08FE819C53775F1
:10434000000013058550EFC07FF737750000130597
:10435000C54BEFC0BFF66FC06F8683A7418C23AA01
:10436000F1E683473900DCA26DBF83A7818C45BF8E
:1043700083A7818B6DB783A7018C55B73307F900ED
:1043800048233387F600850768A393F7F70F69BFC3
:10439000EFB29FFF2E89B2848145130680031385F7
:1043A00041E7EFC00F839387C4FF938941E7A3825E
:1043B000F900834729001947938641E7F91793F7D6
:1043C000F70F636DF7001D678A071307873EBA97DB
:1043D0009C43828783A7C18B23AAF1E6814713867A
:1043E000F4FF63EAC70403A5018B130680039385DA
:1043F00041E7EFC0EFDC19C53775000013058550A4
:10440000EFC0DFEB3775000013058548EFC01FEBE9
:104410006FB0DFFA83A7418C23AAF1E68347390006
:10442000DCA26DBF83A7818C45BF83A7818B6DB74D
:1044300083A7018C55B73307F90048233387F6006B
:10444000850768A393F7F70F69BFEFB2FFF32E89D3
:10445000B284814513068003138541E7EFB07FF7EF
:104460009387C4FF938941E7A382F900834729001A
:104470001947938641E7F91793F7F70F636DF70034
:104480001D678A0713074740BA979C43828783A713
:10449000C18B23AAF1E681471386F4FF63EAC704C0
:1044A00003A5018B13068003938541E7EFC04FD12D
:1044B00019C53775000013058550EFC03FE037750B
:1044C000000013058545EFC07FDF6FB03FEF83A786
:1044D000418C23AAF1E683473900DCA26DBF83A794
:1044E000818C45BF83A7818B6DB783A7018C55B79E
:1044F0003307F90048233387F600850768A393F74D
:10450000F70F69BFEFB25FE82E89B28481451306C9
:104510008003138541E7EFB0DFEB9387C4FF9389F6
:1045200041E7A382F900834729001947938641E7B1
:10453000F91793F7F70F636DF7001D678A071307E5
:104540000742BA979C43828783A7C18B23AAF1E6CF
:1045500081471386F4FF63EAC70403A5018B1306A2
:104560008003938541E7EFC0AFC519C537750000DB
:1045700013058550EFC09FD4377500001305454DD6
:10458000EFC0DFD36FB09FE383A7418C23AAF1E68E
:1045900083473900DCA26DBF83A7818C45BF83A709
:1045A000818B6DB783A7018C55B73307F90048237A
:1045B0003387F600850768A393F7F70F69BFEFB25B
:1045C000BFDC2E89B284814513068003138541E741
:1045D000EFB03FE09387C4FF938941E7A382F900DE
:1045E000834729001947938641E7F91793F7F70F97
:1045F000636DF7001D678A071307C743BA979C438B
:10460000828783A7C18B23AAF1E681471386F4FF33
:1046100063EAC70403A5018B13068003938541E772
:10462000EFC00FBA19C53775000013058550EFC0EC
:10463000FFC83775000013050547EFC03FC86FB0CE
:10464000FFD783A7418C23AAF1E683473900DCA278
:104650006DBF83A7818C45BF83A7818B6DB783A76F
:10466000018C55B73307F90048233387F6008507D7
:1046700068A393F7F70F69BFB7070020142103C79A
:10468000071A639AE6009387071A08319C331D8D39
:1046900013351500828001458280C16769768146A5
:1046A000FD1705061397060141836364B7003E8535
:1046B00082803307D5001823B98F214713F81700DC
:1046C000858363050800B18FC207C1837D17420748
:1046D00041836DF78506F9B7EFB21FCB3704002091
:1046E00013040418AA89AE84328A13090402983488
:1046F0001C406317F7005C405286A6854E85829762
:104700002104E31624FF6FB07FCBEFB2FFC737045D
:10471000002013040415AA89AE84328A1309040305
:10472000D8341C406317F7005C405286A6854E853E
:1047300082972104E31624FF6FB05FC8EFB27FC3F6
:1047400041112A8BEF00007845C97945EFD08FC918
:104750001306200381451385C1DD9389C1DDEFB0C8
:104760005FC7014981440144894B938AC1DD130C21
:1047700000038D4D938C19005A85EF00A0782DCD44
:104780005A85EF00A075137DF50FB38789001306D6
:1047900014002380A70163037601DDC84E8532C66D
:1047A000EFF09FED324609E92286E6854E85EF104F
:1047B000405DE3738CFC89A0A9476304F60063FCA9
:1047C0009B0883C79A00638187091307100A638ACD
:1047D000E7029387070393F7F70F05476374F7061C
:1047E000A68763F37401894793F4F70F75BF938528
:1047F000C1DD5A85EFF05FEE41016FB05FBB3284DF
:104800004DBF6949B1476303F606E31A26FF9305D6
:10481000D6FF93F5F50F4E8532C6EFF01FE83387CC
:104820008A008347E7FF0347F7FF3246A207D98F85
:104830006395A700D947E30CFDFAA687E3F6B4FB1E
:104840008D475DB739497DBFB147E310F6FC19A824
:10485000A947E308F6F6B147E319F6FA83C79A00C9
:10486000E39587FB03C9BA0006093D09314429B71E
:10487000EFB23FB04111AA8BEF00C064630805108E
:104880002945EFD02FB69389C1DD1306200381455A
:104890001385C1DDEFB0FFB3014401498144138AA0
:1048A000C1DD930C0003138D49008D4D138B19004E
:1048B0005E85EF00206579C95E85EF002062937701
:1048C000F50F338799003EC61CA3138C1400914743
:1048D0006304FC00630209124E85EFF0FFD909E979
:1048E0002686DA854E85EF10C049E3F39CFC79A853
:1048F00083462A001D461387F6FF1377F70FE361FF
:10490000E6FE639BB60103473A0019C76D1713779C
:10491000F70F9147E3E6E7FC19476305EC0005470D
:10492000637A27016A85EFF03FD509E5E31A09FAB2
:1049300005497DB739476305EC0009476374270DC6
:104940000347DA00630D9709C1466306D70493064F
:10495000000A630DD7089306100A6302D7081307ED
:1049600007031377F70F854663F2E6080947CA87FE
:104970006373E900894713F9F70F9DB749440DA008
:1049800022869385C1DD5E85EFF03FD841016FB08F
:104990001FA2E28499BF4947630EEC06E31B8CFE1D
:1049A000930584FF93F5E50F6A85EFF01FCF33077A
:1049B0009A008347D7FF8346E7FFA207D58F639B03
:1049C000A7000347F7FFD9476316F7003247DD47D3
:1049D000E308F7FACA87E370B9FB8D4769BF494717
:1049E0005944E31DECFAC9445944D9B54947E30792
:1049F000ECF8E2844944D5BD1947E305ECF23947A8
:104A0000E300ECF44947E31BECF88346DA00414746
:104A1000E396E6F803440A0183471A01C9442204D5
:104A20005D8C2D04060469B5EFB2BF97184183A7CA
:104A3000418C2A846318F7005C2115476397E702CD
:104A4000EF00B0728144377900005C3063CAF4042F
:104A50003775000013058557EFC05F86503008405A
:104A60009305640065266FB01F9619476395E700AC
:104A7000EF005073C1BF1D476395E700EF0030762C
:104A8000D1B721476395E700EF00107965BF25474F
:104A90006395E700EF00F05475B7EF0050595DB72C
:104AA000B3079400EC23130589558504EFC01F81DB
:104AB00069BFEFB27F8D03A5418BEFF03FC803A51F
:104AC000818BEFF0BFC703A5C18BEFF03FC703A5F4
:104AD000018CEFF0BFC603A5418CEFF03FC603A5E4
:104AE000818CEFF0BFC503A5C18CEFF07FD81545D1
:104AF000EFD04F8FC9B7EFB2DF8AB774000013064B
:104B000040068145138501E1EFB0BF8C03A5018B01
:104B1000FD5613064006938501E1EFB09FF2138521
:104B2000C456EFC0AFF9138501E1EFF0FFEFC1BF4D
:104B3000EFB23F87B755000037750000D1470947EE
:104B4000930600200146938525AB1305C555EFC09C
:104B50005FF719C1EFD0AF8E6FB0FF86EFB27F84E1
:104B6000B755000037750000D1470D479306002068
:104B70000146938565AF13054556EFC09FF419C1F3
:104B8000EFD0EF8B6FB03F84EFB2BF81377500007D
:104B900081465146930540061305C557EFB05FDACD
:104BA00023A8A18A3335A0006FB0FF8111CD1C214D
:104BB00089CFEFB20FFF484193F5F50FEF00D00614
:104BC00085473E856FB03F8081473E858280EFB24A
:104BD0004FFD370400209307041B81441304041B7A
:104BE0001D47D443639EA60C960433099400834763
:104BF000090095E71385C4002295EFE0EFEA8327CB
:104C00004900372700409306078003258900639CED
:104C1000D700EF003004B3079400054798A333058D
:104C200094006FB04FFA930607C06395D700EF006A
:104C3000500ED5B7B7460040938606406395D7001F
:104C4000EF001019C9BF6395E700EF009024E1B7AA
:104C500037570040930607806398D704EF00D04091
:104C60008327C90181E7EF00903C75B7154763952D
:104C7000E700EF00904F45B719476395E700EF0055
:104C8000705251BF1D476395E700EF00505561B763
:104C900021476395E700EF003058B5BF2547E39CF7
:104CA000E7F6EF00103485BF6395E700EF00B063CF
:104CB0009DB7130707C0E390E7F6EF009059A1BF37
:104CC000850493870702E39EE4F0014599BFEFB2A4
:104CD0004FED370400201304041B4840130600085E
:104CE0009385C1EAEFF0BFEE23AAA18A48501306CC
:104CF00000089385C1F2EFF09FED23ACA18A6840D4
:104D0000130600089385C1FAEFF07FEC23AEA18A69
:104D10006850130600089385C102EFF05FEB23A0F3
:104D2000A18C03254408130600089385C10AEFF0FF
:104D30001FEA23A2A18C0325440A130600089385C9
:104D4000C112EFF0DFE823A4A18C0325440C130665
:104D500000089385C11AEFF09FE723A6A18C0145B7
:104D60006FB06FE6EFB2EFE385451145EFE0CFBCE2
:104D70006FB06FE5EFB2EFE281451145EFE0CFBBD9
:104D80006FB06FE4EFB2EFE185451545EFE0CFBAC4
:104D90006FB06FE3EFB2EFE081451545EFE0CFB9BB
:104DA0006FB06FE2EFB2EFDF85456145EFE0CFB85E
:104DB0006FB06FE1EFB2EFDE81456145EFE0CFB755
:104DC0006FB06FE0EFB2EFDD854513053002EFE025
:104DD000AFB66FB04FDFEFB2CFDC814513053002C5
:104DE000EFE08FB56FB02FDEEFB2AFDB8545130577
:104DF0007003EFE06FB46FB00FDDEFB28FDA814573
:104E000013057003EFE04FB36FB0EFDBEFB2CFD716
:104E100003A7418B2A842E8AB2891389418B63129E
:104E2000A702EFF03FF4814463C9340583270900EA
:104E3000639E8704EFF01FF40545EFC0BFDA6FB043
:104E4000EFD783A7818B6395A700EFF0BFF3E1BF96
:104E500083A7C18B6395A700EFF0DFF4E9B783A7C1
:104E6000018C6395A700EFF0FFF575BF83A7418C18
:104E7000E39BA7FAEFF05FF77DB7B3079A0083854E
:104E8000070022858504EFF07FD279BF83A7818B4D
:104E900063958700EFF01FF045B783A7C18B63953B
:104EA0008700EFF03FF149BF83A7018C639587002E
:104EB000EFF07FF251B783A7418CE39F87F6EFF0C5
:104EC000DFF39DBF814709C91821814711C75C499C
:104ED000084D898FB337F0003E858280EFB26FCCEA
:104EE00041112A84A3070100EFF0DFFD19C59305E6
:104EF000F1001305C400EFE0EFBE0305F10041012E
:104F00006FB06FCCEFB2EFC93105EFE00FC06FB0FB
:104F10008FCBB7F7FF1F03A5477082805841032846
:104F200005004C4537060140930706403E979346DF
:104F3000F8FFB1C583250640F58D2320B640D04348
:104F4000F18ED4C31443B3E6060114C3184190474D
:104F50009346F7FF758E90C7D047F18ED4C714459E
:104F600041466399C6009447D98E94C7D447558F5C
:104F7000D8C78280B6979443558F98C382801C43CC
:104F8000F58F1CC38280B70701401387074083A7B2
:104F90000740584B698F09C77D8D3335A00082804B
:104FA00001458280B707014023AAA74082809C4523
:104FB00013F7070113F8F70001C7D8413368E80079
:104FC0008E2113F7F50F39C318418146854E3D4FA9
:104FD000930F800293028004214E3396DE00B3F8D3
:104FE000C500631116039398260033131F01134362
:104FF000F3FF3377E300B318180133E7E800639F4A
:10500000F70550C98506E39AC6FD18C11307F00FCE
:105010006375B70454412146854E3D4F930F80027E
:1050200093028004414EB398CE0033F7150163928A
:10503000E8021317260001173313EF001343F3FFA1
:10504000B376D3003317E800D98E639DF701232A86
:1050500015010506E319C6FD54C18280E39457FA91
:1050600010C94DB7E39757FE23281501DDB7084552
:105070006D8D3335A000828019C20CC982804CC965
:10508000828013F7C50F93F73500B7050140BA9535
:1050900094458A073D473317F7001347F7FF758F8D
:1050A00098C598453315F500598D88C5828003A7AA
:1050B000018D894710216311F70214318D4763ED8B
:1050C000D7003C219A0637E700E09607D58F93F783
:1050D000F70F32972300F740544105479357560086
:1050E0003317C70089CA938707048A07B7E600E029
:1050F000B69798C3828093870706C5BF37170240CB
:105100005C439146B18B6385D700A1466382D70685
:10511000B7177A00938707201CC1371602405C42FC
:1051200037070020130707299183BD8BBA97942373
:105130001C41B3D7D7005CC15442A1829D8ABA9664
:105140009422B3D6D70014C55442AD829D8A3697B7
:105150001823B3D7E7005CC55842398393763700EC
:105160001387418036971823B3D7E7021CC9828082
:105170005C435843C166C983758FB7F6FF1F83A68A
:10518000C670BD8B89071396160163480600C54695
:1051900001466392D702C94739A88946638FD7026F
:1051A000BD46638ED702C146638ED702C54601460F
:1051B0006393D700C1471DEF37470240032707809D
:1051C000418B05C737177A0013070720B307F7028B
:1051D0001CC121D61C41858381B701466DBF0546A0
:1051E000B547D1BF0146BD47F9B737173D00130793
:1051F0000790E9BFB7150240D8559316F700D85568
:1052000063DF060411833D8B9306170037177A007E
:10521000130707203357D70218C1D455A182BD8A7E
:105220008DE295463307D702058318C13717024030
:10523000585714413D8B050733D7E60218C1184172
:1052400071B785456394B600E546E9BFBD456396F1
:10525000B600D1463387E602C9BF8906E5BF3D8B5C
:105260009306170037177A00130707203357D70222
:10527000F1B799C5371702401C4F5D8D08CF82806A
:10528000B7170240984F1345F5FF798D88CF82807C
:1052900099C5371702405C4F5D8D48CF8280B717A4
:1052A0000240D84F1345F5FF798DC8CF8280EFB209
:1052B0004F8F1629F577FD17F58FF621DA257971CD
:1052C000D58F1EA95625FD779387379FF58FD62159
:1052D0002A842EC6D58F9625D58FB625D58F5EA567
:1052E0005E29C207C18393F7F7CFD98F5EA96808FB
:1052F000EFF0DFE0B747014093870780B245631EB8
:10530000F402A2576547B387E70298419306400627
:105310000A07B3D7E70233D7D702B3F7D70212078A
:10532000920793872703B3D7D702BD8BD98FC207C4
:10533000C1831EA445616FB00F899257E1B791C533
:105340005E250967D98F5EA582805A25F977FD17FA
:10535000F98FD5BF13F7F50F85471583B395B700C0
:105360006319F7009307C500984301CED98D8CC30C
:105370008280894693074501E318D7FE930705010C
:10538000E5B793C5F5FFF98DDDB793F5F51F4EA190
:1053900082804A211375F51F82800A216D8D333575
:1053A000A000828013F7F50F85461583B397B600EA
:1053B0006311D7025A25F98F1A210145420741830B
:1053C00081CB0545A181B315B5006D8F3335E00064
:1053D000828089466314D7001A29F1BF5A29E1BF98
:1053E000A1818547B397B70093C7F7FFC207C18371
:1053F0001EA18280EFA2FFFA85450945EFD0DFD3D9
:105400006FA07FFCEFA2FFF981450945EFD03FD1A6
:10541000EFF05FFE6FA03FFBEFA2BFF881450545AF
:10542000EFD0FFCF6FA03FFAEFA2BFF72A84EFF0D3
:10543000DFF5930500082285EFF03FF67DD96FA0D8
:105440009FF8EFA21FF6814513056002EFD0DFCE73
:105450006FA07FF7EFA2FFF479712A84814511458F
:10546000EFD0FFCB81451145EFD01FCD814513050E
:105470006002EFD0DFCAEFF0DFFC85454145EFF079
:105480005FDF854513050004EFF09FE08547FC8250
:105490008D44E1474C083715014026CC3ECEEFF055
:1054A0001FB18947FC824C089147371501403ECE19
:1054B000EFF0FFAF22D0372400400C10B7070C00EC
:1054C000130504803ED402D223160102EFF03FDE22
:1054D000930770357C86680085473EC84487EFF0A7
:1054E0001FBD05461305048093055052EFF09FE65B
:1054F000854513050480EFF09FE445616FA0BFEC84
:10550000EFA23FEA814513057002EFD0FFC26FA002
:105510009FEBEFA21FE979712A8481451545EFD0F1
:105520001FC081451545EFD03FC18145130570026D
:10553000EFD0FFBEEFF0DFFC85454145EFF07FD3B4
:10554000854513050008EFF0BFD49147FC828D44D8
:10555000E1474C083715014026CC3ECEEFF03FA581
:10556000A147FC824C089147371501403ECEEFF031
:105570001FA422D0372400400C10B7070C001305DD
:1055800004C03ED402D223160102EFF05FD293078B
:1055900080357C86680085473EC84487EFF03FB180
:1055A0000546130504C093055052EFF0BFDA854558
:1055B000130504C0EFF0BFD845616FA0DFE0EFA294
:1055C0005FDE814513058002EFD01FB76FA0BFDFFC
:1055D000EFA23FDD79712A8981456145EFD03FB463
:1055E00081456145EFD05FB5814513058002EFD05D
:1055F0001FB3EFF0DFFC85451145EFF09FC78545F0
:1056000037050200EFF0DFC8371401409147FC82F4
:105610008D44E1474C081305048026CC3ECEEFF0C4
:105620001F99A147FC824C089147130504803ECE88
:1056300037440040EFF0BF970C10B7070C0013057C
:1056400004404AD03ED402D223160102EFF03FC6F6
:10565000930760337C86680085473EC84487EFF037
:105660001FA505461305044093055052EFF09FCE49
:10567000854513050440EFF09FCC45616FA0BFD472
:10568000EFA23FD2854513059002EFD0FFAA6FA08D
:105690009FD3EFA21FD17971AA84814513053002EF
:1056A000EFD0FFA7814513053002EFD0FFA8814559
:1056B00013059002EFD0BFA6EFF09FFC8545414552
:1056C000EFF03FBB854513050010EFF07FBCC147ED
:1056D0000D44FC824C08E1473715014022CC3ECEF8
:1056E000EFF0FF8C93070002FC824C0891473715BE
:1056F00001403ECEEFF0BF8B0C10B7070C003725F2
:10570000004026D03ED402D223160102EFF03FBA69
:10571000930790357C86680085473EC84087EFF048
:105720001F9905469305505237250040EFF09FC260
:10573000854537250040EFF09FC045616FA0BFC889
:10574000EFA23FC685451305A002EFD0FF9E6FA0D4
:105750009FC7EFA21FC581451305A002EFD0DF9DB3
:105760006FA07FC6EFA2FFC385451305B002EFD03F
:10577000BF9C6FA05FC5EFA2DFC281451305B002D9
:10578000EFD09F9B6FA03FC4EFA2BFC1854513051B
:10579000C002EFD07F9A6FA01FC3EFA29FC08145C8
:1057A0001305C002EFD05F996FA0FFC1EFA27FBFCA
:1057B00085451305D002EFD03F986FA0DFC0EFA260
:1057C0005FBE81451305D002EFD01F976FA0BFBF0A
:1057D000EFA23FBD85451305E002EFD0FF956FA016
:1057E0009FBEEFA21FBCEFF0DFF6EFF0DFF8EFF0A7
:1057F000DFFAEFF0DFFCEFF0BFFD85451305800316
:10580000EFD09F93814513059003EFD0FF9285451C
:105810001305A003EFD05F926FA0FFBAEFA27FB88D
:1058200081451305E002EFD03F916FA0DFB9EFA2F1
:105830005FB7EFF01FF2EFF01FF4EFF01FF6EFF09D
:105840001FF8EFF0BFFD814513058003EFD0DF8E19
:10585000814513059003EFD03F8E81451305A003CA
:10586000EFD09F8D6FA03FB6EFA2BFB37971AA842E
:1058700081451305A002EFD09F8A81451305B00230
:10588000EFD0FF8981451305C002EFD05F898145C4
:105890001305D002EFD0BF8881451305E002EFD099
:1058A0001F88814513057003EFD07F87814513055D
:1058B0007003EFD07F88814513058003EFD03F86CA
:1058C000814513059003EFD09F8581451305A00303
:1058D000EFD0FF84EFF0BFF585452145EFF07F99CC
:1058E000854537050400EFF0BF9A93070040FC821E
:1058F000371401408D473ECC4C08E147130504C0E6
:105900003ECEEFF0CFEA856793870780FC824C0894
:105910009147130504C03ECE37540040EFF02FE905
:105920000C10B7070C001305048026D03ED402D219
:1059300023160102EFF0BF97930770137C8685470B
:105940005C87680085473EC8EFF06FF60546130593
:10595000048093055052EFF0FF9F854513050480A6
:10596000EFF0FF9D45616FA01FA6EFA29FA3EFF090
:105970003FDDEFF05FE0EFF05FE2EFF05FE4EFF0CC
:10598000FFE9814513058003EFD00FFB8145130527
:105990009003EFD06FFA81451305A003EFD0CFF944
:1059A0006FA07FA2EFA2FF9FEFF0BFDAEFF09FDBC7
:1059B000EFF0BFDEEFF0BFE0EFF05FE685451305E7
:1059C0008003EFD06FF7814513059003EFD0CFF63A
:1059D00081451305A003EFD02FF66FA0DF9EEFA245
:1059E0005F9CEFF01FD7EFF01FD9EFF0FFD9EFF07A
:1059F0001FDDEFF0BFE2854513058003EFD0CFF345
:105A0000854513059003EFD02FF381451305A003BF
:105A1000EFD08FF26FA03F9BEFA2BF98EFF07FD344
:105A2000EFF07FD5EFF07FD7EFF05FD8EFF01FDF1B
:105A3000814513058003EFD02FF0814513059003B6
:105A4000EFD08FEF85451305A003EFD0EFEE6FA0E9
:105A50009F97EFA21F9579712A8485454145EFF004
:105A60005F81854537050800EFF09F82930700406E
:105A7000FC828D44E1474C083715014026CC3ECED0
:105A8000EFF0EFD2856793870780FC824C0891473F
:105A9000371501403ECEEFF08FD122D03754004071
:105AA0000C10B7070C00130504C03ED402D2231615
:105AB0000102EFF0CFFF930740347C8668008547F2
:105AC0003EC84487EFF0AFDE0546130504C09305DA
:105AD0005052EFF03F888545130504C0EFF03F8634
:105AE00045616FA05F8EEFA2DF8B7971AA84854537
:105AF0004145EFF00FF8854513050002EFF06FF711
:105B0000854537051000EFF0AFF885670D44FC823E
:105B10004C08E1473715014022CC3ECEEFF02FC9AB
:105B2000914737150140FC824C0891471305054009
:105B30003ECEEFF0CFC70C10B7070C003755004032
:105B400026D03ED402D223160102EFF04FF693077F
:105B500050347C86680085473EC84087EFF02FD5DB
:105B600005469305505237550040EFF0AFFE85458E
:105B700037550040EFF0AFFC45616FA0DF84411165
:105B800022C6374400409305505213050440EFF0FD
:105B90007F8115C513050440EFF0AFFF9375F50F36
:105BA0002384B18E03A5C18B1C4D10495449850730
:105BB000B3E7C7026385D7003105EFD0EFEF32447A
:105BC000410173002030411122C637540040930533
:105BD000505213050480EFF0EFFC15C51305048047
:105BE000EFF02FFB9375F50F2386B18E03A5418C43
:105BF0001C4D104954498507B3E7C7026385D70098
:105C00003105EFD06FEB3244410173002030411178
:105C100022C63754004093055052130504C0EFF0DC
:105C20006FF815C5130504C0EFF0AFF69375F50FC7
:105C3000238AB18C03A5818C1C4D104954498507DA
:105C4000B3E7C7026385D7003105EFD0EFE63244F2
:105C50004101730020309305505237550040EFF05A
:105C60006FF415C537550040EFF0AFF29375F50F9F
:105C7000238CB18C03A5C18C1C4D10495449850758
:105C8000B3E7C7026385D7003105EFD0EFE27300B9
:105C90002030411122C6372400409305505213058D
:105CA0000480EFF02FF015C513050480EFF06FEEC0
:105CB0009375F50F238EB18C03A5418B1C4D1049B4
:105CC00054498507B3E7C7026385D7003105EFD094
:105CD000AFDE3244410173002030411122C6372427
:105CE000004093055052130504C0EFF0AFEB15C50B
:105CF000130504C0EFF0EFE99375F50F2380B18E23
:105D000003A5818B1C4D104954498507B3E7C70291
:105D10006385D7003105EFD02FDA3244410173009B
:105D200020309305505237250040EFF0AFE715C5FE
:105D300037250040EFF0EFE59375F50F2382B18E24
:105D400003A5018C1C4D104954498507B3E7C702D0
:105D50006385D7003105EFD02FD67300203001477F
:105D60006314E60001458280B307E5000507B386AA
:105D7000E5009C2383C6F6FFE384D7FE3385D74036
:105D80008280B3C7A5008D8B3307C50081E78D479F
:105D900063EDC700AA87637EE50894218507850522
:105DA000A38FD7FEE3EBE7FE828093763500AA87C8
:105DB00089CA942185078505A38FD7FE93F63700FE
:105DC000C5BF9376C7FF138606FE63F0C70683A39D
:105DD000050083A2450083AF850003AFC50083AEF5
:105DE000050103AE450103A3850183A8C501938581
:105DF000450223A0770003A8C5FF23A2570023A4D0
:105E0000F70123A6E70123A8D70123AAC70123ACE2
:105E1000670023AE17019387470223AE07FF75B7CC
:105E200090419107910523AEC7FEE3EBD7FEE3E671
:105E3000E7F68280AA8798239386170009EB8505E9
:105E400003C7F5FF8507A38FE7FE75FB8280B68742
:105E5000DDB7AA87982185078505A38FE7FE7DFB1F
:105E60008280AA87850703C7F7FF6DFF3385A740A8
:105E70007D15828015C27D160147B307E500B38604
:105E8000E5009C2394226396D7006304C7000507AE
:105E9000EDF73385D7408280014582806469000038
:105EA00078690000886900009C690000A86900000A
:105EB000B4690000B8690000C8690000D869000032
:105EC000E0690000F4690000046A00000C6A000048
:105ED000186A0000246A0000386A0000406A000066
:105EE000506A0000606A0000786A00006D61696EA7
:105EF00000000000546F20696E697469616C697AF2
:105F000065206465766963653A2573206661696C0E
:105F100065642E20546865206572726F7220636F0D
:105F200064652069732025640A0000007469646C4C
:105F300065000000000001000200010003000100F4
:105F40000200010004000100020001000300010042
:105F50000200010005000100020001000300010031
:105F60000200010004000100020001000300010022
:105F70000200010006000100020001000300010010
:105F80000200010004000100020001000300010002
:105F900002000100050001000200010003000100F1
:105FA00002000100040001000200010003000100E2
:105FB00002000100070001000200010003000100CF
:105FC00002000100040001000200010003000100C2
:105FD00002000100050001000200010003000100B1
:105FE00002000100040001000200010003000100A2
:105FF0000200010006000100020001000300010090
:106000000200010004000100020001000300010081
:106010000200010005000100020001000300010070
:106020000200010004000100020001000300010061
:1060300002000100303132333435363738394142CD
:1060400043444546000000000A205C207C202F0AC3
:10605000000000002D205254202D2020202020540C
:106060006872656164204F7065726174696E672043
:1060700053797374656D0A00417567203139203298
:1060800030323400202F207C205C2020202020254E
:10609000642E25642E2564206275696C6420257346
:1060A0000A0000002032303036202D2032303139C5
:1060B00020436F7079726967687420627920727406
:1060C0002D746872656164207465616D0A0000005A
:1060D000284E554C4C290000303132333435363798
:1060E000383961626364656600000000746F746132
:1060F0006C206D656D6F72793A2025640A0000008E
:1061000075736564206D656D6F7279203A20256422
:106110000A0000006D6178696D756D20616C6C6FAF
:106120006361746564206D656D6F72793A202564D2
:106130000A0000006C697374206D656D6F727920C0
:10614000757361676520696E666F726D6174696FE2
:106150006E0000006C6973745F6D656D0000000077
:10616000746F2066726565206120626164206461DD
:10617000746120626C6F636B3A0A00006D656D3A62
:10618000203078253038782C207573656420666C53
:1061900061673A2025642C206D6167696320636F15
:1061A00064653A203078253034780A00686561707B
:1061B000000000006D656D20696E69742C206572A9
:1061C000726F7220626567696E20616464726573C4
:1061D0007320307825782C20616E6420656E6420F1
:1061E0006164647265737320307825780A0000005A
:1061F0001B5B324A1B5B48002D2D46756E6374692C
:106200006F6E204C6973743A0A0000005F5F0000F3
:10621000252D313673202D2D2025730A0000000016
:106220006465766963650000252D2A2E7320202081
:10623000202020202020747970652020202020201C
:1062400020202072656620636F756E740A0000005E
:10625000202D2D2D2D2D2D2D2D2D2D2D2D2D2D2D7B
:106260002D2D2D2D2D202D2D2D2D2D2D2D2D2D2D6B
:106270000A000000252D2A2E2A7320252D32307386
:1062800020252D38640A00006576656E74000000D4
:10629000252D2A2E73202020202020736574202095
:1062A000202073757370656E642074687265616414
:1062B0000A00000020202D2D2D2D2D2D2D2D2D2DD2
:1062C000202D2D2D2D2D2D2D2D2D2D2D2D2D2D0A2E
:1062D00000000000252D2A2E2A732020307825303A
:1062E000387820253033643A00000000252D2A2E0E
:1062F0002A73202030782530387820300A000000BA
:106300006D61696C626F7800252D2A2E7320656E91
:106310007472792073697A652073757370656E6421
:10632000207468726561640A00000000202D2D2D24
:106330002D20202D2D2D2D202D2D2D2D2D2D2D2DB4
:106340002D2D2D2D2D2D0A00252D2A2E2A732025A9
:106350003034642020253034642025643A00000065
:10636000252D2A2E2A732025303464202025303410
:10637000642025640A0000006D736771756575659A
:1063800000000000252D2A2E7320656E747279207E
:1063900073757370656E64207468726561640A0059
:1063A000202D2D2D2D20202D2D2D2D2D2D2D2D2D44
:1063B0002D2D2D2D2D0A0000252D2A2E2A73202566
:1063C000303464202025643A00000000252D2A2E58
:1063D0002A732025303464202025640A0000000040
:1063E0006D75746578000000252D2A2E73202020FD
:1063F0006F776E65722020686F6C642073757370A0
:10640000656E64207468726561640A00202D2D2D0C
:106410002D2D2D2D2D202D2D2D2D202D2D2D2D2DC6
:106420002D2D2D2D2D2D2D2D2D0A0000252D2A2E23
:106430002A7320252D382E2A7320253034642025F8
:10644000640A000073656D6170686F72650000001A
:10645000252D2A2E73207620202073757370656E8B
:1064600064207468726561640A000000202D2D2D7F
:10647000202D2D2D2D2D2D2D2D2D2D2D2D2D2D0A7C
:1064800000000000252D2A2E2A7320253033642099
:1064900025643A00252D2A2E2A73202530336420C6
:1064A00025640A007468726561640000252D2A2E37
:1064B00073207072692020737461747573202020BA
:1064C00020202073702020202020737461636B20B3
:1064D00073697A65206D61782075736564206C65D9
:1064E0006674207469636B20206572726F720A0093
:1064F000202D2D2D20202D2D2D2D2D2D2D202D2D00
:106500002D2D2D2D2D2D2D2D202D2D2D2D2D2D2DC8
:106510002D2D2D20202D2D2D2D2D2D20202D2D2DDF
:106520002D2D2D2D2D2D2D202D2D2D0A000000007F
:10653000252D2A2E2A7320253364200020726561C0
:1065400064792020000000002073757370656E640C
:106550000000000020696E69742020200000000007
:1065600020636C6F736520200000000020307825C8
:106570003038782030782530387820202020253099
:1065800032642525202020307825303878202530A9
:1065900033640A0074696D6572000000252D2A2E8F
:1065A000732020706572696F6469632020207469AC
:1065B0006D656F757420202020202020666C616737
:1065C0000A000000202D2D2D2D2D2D2D2D2D2D20BF
:1065D0002D2D2D2D2D2D2D2D2D2D202D2D2D2D2DF8
:1065E0002D2D2D2D2D2D0A00252D2A2E2A732030FC
:1065F0007825303878203078253038782000000031
:106600006163746976617465640A0000646561633E
:10661000746976617465640A0000000063757272C3
:10662000656E74207469636B3A3078253038780A67
:10663000000000006C69737420616C6C2073796DCC
:10664000626F6C20696E2073797374656D00000051
:106650006C697374000000006C6973742064657663
:1066600069636520696E2073797374656D0000003D
:106670005F5F636D645F6C6973745F6465766963A3
:10668000650000006C697374206465766963652039
:10669000696E2073797374656D0000006C697374A2
:1066A0005F646576696365006C6973742074696DF5
:1066B000657220696E2073797374656D0000000047
:1066C0005F5F636D645F6C6973745F74696D65723D
:1066D000000000006C6973742074696D6572206934
:1066E0006E2073797374656D000000006C697374BB
:1066F0005F74696D657200006C697374206D6573F9
:106700007361676520717565756520696E207379A1
:106710007374656D000000005F5F636D645F6C699A
:1067200073745F6D73677175657565006C697374FB
:10673000206D657373616765207175657565206986
:106740006E2073797374656D000000006C6973745A
:106750005F6D736771756575650000006C697374B2
:10676000206D61696C20626F7820696E2073797387
:1067700074656D005F5F636D645F6C6973745F6DFA
:1067800061696C626F7800006C697374206D616977
:106790006C20626F7820696E2073797374656D0068
:1067A0006C6973745F6D61696C626F7800000000E2
:1067B0006C697374206D7574657820696E207379C7
:1067C0007374656D000000005F5F636D645F6C69EA
:1067D00073745F6D75746578000000006C69737484
:1067E000206D7574657820696E2073797374656D9A
:1067F000000000006C6973745F6D7574657800004B
:106800006C697374206576656E7420696E20737987
:106810007374656D000000005F5F636D645F6C6999
:1068200073745F6576656E74000000006C69737444
:10683000206576656E7420696E2073797374656D5A
:10684000000000006C6973745F6576656E7400000B
:106850006C6973742073656D6170686F726520690F
:106860006E2073797374656D000000005F5F636D67
:10687000645F6C6973745F73656D00006C69737439
:106880002073656D6170686F6E6520696E20737925
:106890007374656D000000006C6973745F73656DDF
:1068A000000000006C697374207468726561640094
:1068B0005F5F636D645F6C6973745F746872656158
:1068C000640000006C697374207468726561640010
:1068D0006C6973745F7468726561640074686520C4
:1068E0007465726D696E616C2073637265656E00AC
:1068F0005F5F636D645F636C6561720074686520DF
:106900007465726D696E616C2073637265656E008B
:10691000636C6561720000007265626F6F74207451
:10692000686520626F617264000000005F5F636DE4
:10693000645F7265626F6F74000000007265626F61
:106940006F742074686520626F61726400000000DB
:106950007265626F6F7400002D00000025730000E7
:106960002F000000436861726163746572204465A2
:106970007669636500000000426C6F636B204465BC
:1069800076696365000000004E6574776F726B2056
:10699000496E746572666163650000004D54442061
:1069A000446576696365000043414E20446576691D
:1069B0006365000052544300536F756E6420446554
:1069C0007669636500000000477261706869632042
:1069D000446576696365000049324320427573005F
:1069E00055534220536C6176652044657669636532
:1069F0000000000055534220486F737420427573A5
:106A00000000000053504920427573005350492044
:106A100044657669636500005344494F20427573AD
:106A200000000000504D2050736575646F20446570
:106A30007669636500000000506970650000000021
:106A4000506F7274616C2044657669636500000064
:106A500054696D65722044657669636500000000C5
:106A60004D697363656C6C616E656F757320446509
:106A70007669636500000000556E6B6E6F776E007F
:106A8000546F6F206D616E792061726773202120D1
:106A90005765206F6E6C79205573653A0A000000C7
:106AA0002573200025733A20636F6D6D616E64203D
:106AB0006E6F7420666F756E642E0A0052542D54EA
:106AC0006872656164207368656C6C20636F6D6DBE
:106AD000616E64733A0A00005F5F636D645F00007B
:106AE000252D313673202D2025730A0052542D5444
:106AF0006872656164207368656C6C2068656C7091
:106B0000000000005F5F636D645F68656C7000008B
:106B100053686F7720746865206D656D6F7279209A
:106B2000757361676520696E207468652073797379
:106B300074656D005F5F636D645F6672656500001C
:106B40004C697374207468726561647320696E2087
:106B50007468652073797374656D00005F5F636DA1
:106B6000645F7073000000006D7368200000000017
:106B700066696E73682000003E00000066696E73EF
:106B8000683A2063616E206E6F742066696E6420BF
:106B90006465766963653A2025730A006E6F206D1F
:106BA000656D6F727920666F72207368656C6C0A10
:106BB00000000000747368656C6C00007368727884
:106BC0000000000008000000256300000825732075
:106BD00020080000082008001B5B324B0D0000005D
:106BE0002573257300000000726561642073746171
:106BF0007475732066726F6D20686172647761725C
:106C0000652070696E00000070696E5265616400F5
:106C100077726974652076616C756520746F206881
:106C2000617264776172652070696E0070696E5779
:106C30007269746500000000736574206861726495
:106C4000776172652070696E206D6F646500000069
:106C500070696E4D6F64650075617274310000007B
:106C600006340000C6330000E8330000843400001E
:106C7000163500007035000001000000160000000D
:106C800002000000170000000400000018000000CF
:106C90000800000019000000100000001A000000A9
:106CA0002000000027000000400000002700000036
:106CB0008000000027000000000100002700000005
:106CC000000200002700000000040000380000005F
:106CD000000800003800000000100000380000002C
:106CE00000200000380000000040000038000000D4
:106CF0000080000038000000FFFFFFFF00000000E0
:106D000000000000000000000100000078330000D7
:106D10000018014004000000020000007833000069
:106D20000018014008000000030000007833000054
:106D3000001801401000000004000000783300003B
:106D4000001801402000000005000000783300001A
:106D50000018014040000000FFFFFFFF000000009E
:106D60000000000000000000070000006833000081
:106D700000100140002000000800000068330000FF
:106D800000100140004000000900000068330000CE
:106D90000010014000800000FFFFFFFF0000000026
:106DA0000000000000000000FFFFFFFF00000000E7
:106DB0000000000000000000FFFFFFFF00000000D7
:106DC0000000000000000000FFFFFFFF00000000C7
:106DD0000000000000000000FFFFFFFF00000000B7
:106DE00000000000000000000F00000068330000F9
:106DF0000010014001000000100000006833000096
:106E00000010014002000000110000006833000083
:106E10000010014004000000120000006833000070
:106E20000010014008000000FFFFFFFF000000000D
:106E30000000000000000000FFFFFFFF0000000056
:106E40000000000000000000FFFFFFFF0000000046
:106E50000000000000000000FFFFFFFF0000000036
:106E60000000000000000000170000005833000080
:106E70000008014001000000180000005833000025
:106E80000008014002000000190000005833000013
:106E900000080140040000001A0000005833000000
:106EA0000008014008000000FFFFFFFF0000000095
:106EB0000000000000000000FFFFFFFF00000000D6
:106EC00000000000000000001D000000583300001A
:106ED00000080140100000001E00000058330000B0
:106EE00000080140200000001F000000583300008F
:106EF000000801404000000020000000583300005E
:106F000000080140800000002100000068330000FC
:106F10000010014010000000220000006833000053
:106F20000010014020000000230000004833000052
:106F3000000C014001000000240000004833000064
:106F4000000C014002000000250000004833000052
:106F5000000C01400400000026000000783300000F
:106F60000018014080000000270000007833000076
:106F700000180140000100002800000078330000E4
:106F800000180140000200002900000078330000D2
:106F900000180140000400002A00000078330000BF
:106FA00000180140000800002B00000078330000AA
:106FB00000180140001000002C0000007833000091
:106FC00000180140002000002D0000007833000070
:106FD00000180140004000002E000000783300003F
:106FE00000180140008000002F000000483300001E
:106FF000000C014000040000300000004833000095
:10700000000C014000080000FFFFFFFF000000002F
:107010000000000000000000FFFFFFFF0000000074
:1070200000000000000000003300000048330000B2
:10703000000C014000100000340000004833000044
:10704000000C014000200000350000004833000023
:10705000000C0140004000003600000048330000F2
:10706000000C0140008000003700000036330000B3
:107070000014014000010000380000003633000019
:107080000014014000020000390000003633000007
:1070900000140140000400003A00000036330000F4
:1070A00000140140000800003B00000036330000DF
:1070B00000140140001000003C00000036330000C6
:1070C00000140140002000003D00000036330000A5
:1070D00000140140004000003E0000003633000074
:1070E00000140140008000003F00000068330000F1
:1070F0000010014040000000400000006833000024
:1071000000100140800000004100000068330000D2
:107110000010014000010000420000006833000040
:10712000001001400002000043000000583300003E
:107130000008014000010000440000005833000036
:107140000008014000020000450000005833000024
:107150000008014000040000460000005833000011
:1071600000080140000800004700000058330000FC
:1071700000080140001000004800000058330000E3
:107180000008014000200000FFFFFFFF000000009A
:107190000000000000000000FFFFFFFF00000000F3
:1071A0000000000000000000FFFFFFFF00000000E3
:1071B00000000000000000004C00000058330000F8
:1071C00000080140004000004D000000583300005E
:1071D00000080140008000004E00000068330000FD
:1071E00000100140000400004F0000006833000060
:1071F000001001400008000050000000683300004B
:107200000010014000100000510000003633000063
:10721000001401400100000052000000363300005D
:10722000001401400200000053000000363300004B
:107230000014014004000000540000003633000038
:107240000014014008000000550000003633000023
:10725000001401401000000056000000363300000A
:1072600000140140200000005700000036330000E9
:1072700000140140400000005800000036330000B8
:107280000014014080000000590000004833000055
:10729000000C0140080000005A00000048330000C4
:1072A000000C0140100000005B00000048330000AB
:1072B000000C0140200000005C000000483300008A
:1072C000000C0140400000005D0000004833000059
:1072D000000C014080000000FFFFFFFF00000000E5
:1072E00000000000000000005F00000048330000C4
:1072F000000C014000010000600000004833000065
:10730000000C014000020000610000007833000022
:107310000018014001000000620000007833000006
:107320000018014002000000FFFFFFFF0000000006
:107330000000000000000000FFFFFFFF0000000051
:10734000000000000000000070696E00B43800000A
:10735000823A0000603A00003E3A0000B038000077
:10736000206861726466756C740D0A00204E4D4988
:107370002048616E646C65720D0A00000D0A204D94
:1073800043553A2043483332563330330D0A000018
:1073900020537973436C6B3A202564487A0D0A00B8
:1073A000204368697049443A20253038780D0A0036
:1073B00060420000A0420000B042000068420000AD
:1073C00060420000B6420000BC4200001A430000C8
:1073D0005A4300006A430000224300001A430000A1
:1073E0007043000076430000D443000014440000C2
:1073F00024440000DC430000D44300002A44000081
:10740000304400008E440000CE440000DE44000002
:10741000964400008E440000E4440000EA4400006A
:107420004845000088450000984500005045000090
:10743000484500009E450000A445000002460000AB
:1074400042460000524600000A4600000246000084
:10745000584600005E46000020696E2042726F614F
:1074600064636173745F5363616E200A20000000DF
:1074700020696E20526561645F5265676973746547
:1074800072200A200000000020696E2052656769A2
:107490007374726174696F6E5F7265717565737410
:1074A000200A200020696E2052656D6F74655F555B
:1074B000706772616465200A2000000020696E20F8
:1074C0005570646174655F50726F66696C65200AFF
:1074D0002000000020696E2057726974655F526554
:1074E000676973746572200A2000000020696E20AD
:1074F00053656E736F725F526561645F5265676951
:1075000073746572200A200072745F6D715F736519
:107510006E64204552520A0020696E2053656E73D6
:107520006F725F52656D6F74655F557067726164ED
:1075300065200A200000000020696E2053656E73EC
:107540006F725F5570646174655F50726F66696CCD
:1075500065200A200000000025782000526563762F
:107560000000000073656E64000000000A2053658F
:107570006E642062756666200A00000053656E64C2
:107580005F6D710054610000346100000814000058
:10759000506600003466000002250000706600009E
:1075A00058660000D42300009C660000846600003A
:1075B000D4230000C0660000A86600006824000014
:1075C000EC660000D4660000682400001867000024
:1075D000F86600001E2300004C6700002C670000C6
:1075E0001E230000746700005C670000602200003A
:1075F000A06700008867000060220000C8670000E4
:10760000B0670000DE210000F4670000DC670000C6
:10761000DE21000018680000006800003221000030
:10762000446800002C680000322100006C680000F3
:10763000506800007C200000986800007C68000012
:107640007C200000B0680000A4680000981F0000C3
:10765000D0680000C4680000981F0000F0680000B7
:10766000DC680000EE1E000010690000FC680000ED
:10767000EE1E00002C69000018690000DC1E0000EE
:10768000506900003C690000DC1E0000046B000033
:10769000EC6A00004C250000346B0000106B000009
:1076A000022800005C6B0000406B0000F427000023
:1076B000086C0000E86B0000523100002C6C0000E8
:1076C000106C000038310000506C0000386C000075
:1076D0001E310000D0040000D80400008A330000EE
:1076E00082390000DC04000022280000D4040000DD
:1076F00001000000040000200400002080000000C1
:1077000002000000140000201400002020000000EF
:1077100003000000240000202400002024000000BA
:10772000040000003400002034000020200000008D
:10773000050000004400002044000020300000004C
:107740000600000054000020540000203400000017
:1077500009000000640000206400002044000000D4
:107760000A00000074000020740000202C000000BB
:10777000FFFF00000000000000000000FFFF00000D
:107780000000000000000000FFFF000000000000FB
:1077900000000000FFFF00000000000000000000EB
:1077A000FFFF00000000000000000000FFFF0000DD
:1077B0000000000000000000FFFF000000000000CB
:1077C00000000000FFFF00000000000000000000BB
:1077D000FFFF00000000000000000000FFFF0000AD
:1077E0000000000000000000FFFF0000000000009B
:1077F00000000000FFFF000000000000000000008B
:10780000FFFF00000000000000000000FFFF00007C
:107810000000000000000000FFFF0000000000006A
:1078200000000000FFFF000000000000000000005A
:107830000000000000000000010203040607080920
:1078400030000000BE4500001000000004450000AC
:10785000A00000004A440000A10000009043000086
:10786000D0000000D6420000D10000001C42000001
:107870003000000038410000A1000000604000001E
:10788000D00000007C3F0000D1000000983E0000C6
:10789000534C0000000000000016534C000017007D
:1078A00000000000001800408025000000000000DB
:1078B00000000000000000000000000001000000C7
:1078C00000000000001C00408025000000000000B7
:1078D00000000000000000000000000001000000A7
:1078E000000000000044004080250000000000006F
:1078F0000000000000000000000000000100000087
:107900000000000000200040802500000000000072
:107910000000000000000000000000000100000066
:10792000000000000048004080250000000000002A
:107930000000000000000000000000000000000047
:1079400000000000004C0040802500000000000006
:107950000000000000000000000000000100000026
:10796000000000000050004000C2010000000000C4
:107970000000000000000000000000000100000006
:1079800000000000010203040102030406070809C5
:0879900000D8B8050204060846
:00000001FF
